:100000000C9484170C94AC170C94AC170C94AC178C
:100010000C94AC170C94AC170C94AC170C94CE3514
:100020000C94AC170C94AC170C94AC170C94AC1744
:100030000C94AC170C94AC170C94AC170C94AC1734
:100040000C94AB300C94AC170C9481320C94C832E5
:100050000C94AC170C94AC170C94AC170C94AC1714
:100060000C94AC170C94AC17071B091B091B091B3C
:10007000091B091B091B091B091B091B091B091B60
:10008000F51A091BB91AD71AAB1A2D1A3B1A491AB5
:10009000571A651A731A811A8F1A9D1A091B091BA0
:1000A000091BC91A091BE51A091B091B091B091B96
:1000B000091B091B091B091B091B091B091B091B20
:1000C000091B091B091B091B091B091B091B091B10
:1000D000091B091B091B091B091B091B091B091B00
:1000E000091B091B091B091B091B21192919351992
:1000F00041194B1951195D19671973197B19871922
:1001000091199D19A519AD19B719C319CF19D91985
:10011000E319E919F319FF19091A151A211A6F6B56
:100120003B0077783B0072783B0074783B00676453
:100130003B00646C3B0069733B006F703B00796C63
:100140003B0064653B0061633B0065723B00657387
:100150003B0037333B0063713B0068693B006F65D0
:100160003B00676E3B006F763B00776B3B00736F25
:100170003B0035353B0061743B0064783B006662B0
:100180003B006E6F3B006D793B0076793B00746FEE
:100190003B006F663B0065753B00766C3B00697405
:1001A0003B006D653B0063773B006A613B006F621B
:1001B0003B0064613B00696E3B006F6E3B00626B0D
:1001C0003B00646F3B0061673B00676F3B006174FD
:1001D0003B006B6D3B0073703B0062793B006862D3
:1001E0003B0070613B0064783B0075733B00646CBE
:1001F0003B0067743B00666D3B00616D3B00676EC2
:100200003B0067703B0068663B006C773B006E729A
:100210003B006E773B006F6D3B0072663B00736E78
:100220003B00766C3B00776C3B00796C3B003535CE
:100230003B0061733B001E01220126012A012E01B1
:10024000320136013A013E01420146014A014E01A6
:10025000520156015A015E01620166016A016E0196
:10026000720176017A017E01820186018A018E0186
:10027000920196019A019E01A201A601AA01AE0176
:10028000B201B601BA01BE01C201C601CA01CE0166
:10029000D201D601DA01DE01E201E601EA01EE0156
:1002A000F201F601FA01FE01020206020A020E0242
:1002B000120216021A021E02220226022A022E022E
:1002C0003202746E783B007372693B007173623B5B
:1002D000006162743B007269673B007769723B00A2
:1002E0006D69743B006469643B00756E733B007319
:1002F00068653B00636C723B00616E743B00747216
:10030000783B007073653B00746B733B006E696CE7
:100310003B006D69723B006469723B0078796C3B0D
:100320000074776F3B0071736F3B006665723B0032
:100330006861743B007761723B006872643B006CDB
:1003400074723B0069686D3B0077686F3B006375B2
:100350006C3B007761733B007075743B006275679E
:100360003B006572653B006561723B006F68723BE4
:1003700000626F783B006269673B00616E643B001E
:10038000756E643B006C6F743B0064656D3B00717F
:10039000736C3B0077726B3B0065696E3B00746861
:1003A000653B0071736F3B007369653B0071727050
:1003B0003B0071726F3B0071736B3B006F76763B55
:1003C000007377723B007275663B006C6F733B0085
:1003D000676E643B006169723B0064776E3B006648
:1003E0006F673B006E75723B00626F793B00736113
:1003F000653B0068616D3B006972633B00766F6E20
:100400003B006C6F773B006C65743B007566623B2C
:1004100000746F6F3B006263693B006B65793B0062
:100420007373623B00706B743B00746D773B0064C8
:1004300069653B006461733B006D6E693B007172DE
:100440007A3B007273743B006672713B0075736592
:100450003B0077706D3B0062706D3B006F6E653BDB
:10046000006269743B0073776C3B007270743B00F0
:100470006275673B006F75743B007768793B00716C
:10048000736C3B007668663B0076666F3B0071726A
:100490006D3B007476693B00766C6E3B006C62725B
:1004A0003B006D696E3B006469723B0063666D3BA7
:1004B0000061676E3B0071726E3B007172673B00BA
:1004C00066756E3B0073756E3B00616D703B00712D
:1004D000726C3B006C65643B00616C733B00646153
:1004E000733B006465723B00C202C702CC02D102BA
:1004F000D602DB02E002E502EA02EF02F402F902B0
:10050000FE02030308030D03120317031C03210358
:1005100026032B03300335033A033F034403490307
:100520004E03530358035D03620367036C037103B7
:1005300076037B03800385038A038F039403990367
:100540009E03A303A803AD03B203B703BC03C10317
:10055000C603CB03D003D503DA03DF03E403E903C7
:10056000EE03F303F803FD03020407040C04110473
:1005700016041B04200425042A042F04340439041F
:100580003E04430448044D04520457045C046104CF
:1005900066046B04700475047A047F04840489047F
:1005A0008E04930498049D04A204A704AC04B1042F
:1005B000B604BB04C004C504CA04CF04D404D904DF
:1005C000DE04E30468616E643B00776972653B009A
:1005D000686175733B00746861743B007361736597
:1005E0003B006D616E6E3B00736E6F773B00646124
:1005F00063683B00726F6F663B006371646C3B0025
:100600006D6173743B006C6573653B006D6F737453
:100610003B00776572653B0064616E6E3B0066650A
:10062000696E3B0074656D703B007365656E3B00E1
:10063000726376723B00726376643B0073616D6532
:100640003B007761726D3B00636F6F6C3B00786DB0
:1006500074723B00626F79733B007468656E3B0097
:100660006D6164653B00627563683B007863757318
:100670003B007768656E3B0077726B643B00676593
:1006800062653B00737563683B00666F6E653B0097
:10069000686162653B007265696E3B00676568650D
:1006A0003B007A61686C3B006562656E3B00677277
:1006B00061643B006265656E3B0066616C6C3B008B
:1006C000686F6D653B00636F6E643B0064616E6EC6
:1006D0003B00746869733B00746861743B00647824
:1006E00063633B00657264653B0063616C6C3B0057
:1006F00064696E673B006D6163683B006D6F726596
:100700003B00727474793B00616C736F3B006D69E0
:1007100073743B00637264733B00646F72743B00DC
:1007200064616E6E3B00717565723B006D6F76653E
:100730003B006F7665723B00616265723B006461ED
:1007400073683B00646F63683B00646172633B00E5
:100750006C696B653B00727072743B00696872650E
:100760003B006465696E3B00686F63683B00736BB8
:1007700065643B00736967733B006E65696E3B009F
:100780006D6568723B00667573733B0066756E6BD2
:100790003B0064656E6B3B0064616E6B3B006B728B
:1007A000616E3B006E65696E3B006265616D3B008A
:1007B00069636F6D3B00736173653B007874616CB6
:1007C0003B00777474733B00696E666F3B00626335
:1007D0006E753B00617764683B00696E70743B0026
:1007E0006270736B3B00686F63683B007469656699
:1007F0003B00616265723B006E6F63683B0079612C
:1008000072643B007365656E3B0062616E643B0021
:10081000626572673B006D6565723B007369656771
:100820003B006172726C3B006D6965663B00616400
:1008300065723B007765696E3B0073656B743B00C6
:100840007A61756E3B006B61756D3B007261756D11
:100850003B006A756D703B00C405CA05D005D6051E
:10086000DC05E205E805EE05F405FA0500060606D6
:100870000C06120618061E0624062A063006360640
:100880003C06420648064E0654065A0660066606B0
:100890006C06720678067E0684068A069006960620
:1008A0009C06A206A806AE06B406BA06C006C60690
:1008B000CC06D206D806DE06E406EA06F006F60600
:1008C000FC06020708070E0714071A072007260769
:1008D0002C07320738073E0744074A0750075607D8
:1008E0005C07620768076E0774077A078007860748
:1008F0008C07920798079E07A407AA07B007B607B8
:10090000BC07C207C807CE07D407DA07E007E60727
:10091000EC07F207F807FE0704080A081008160893
:100920001C08220828082E0834083A0840084608FF
:100930004C085208676C617562653B006E696368BC
:10094000743B00696D6D65723B0077696564657223
:100950003B0066756E6B656E3B00616E74656E6E16
:10096000653B006469706F6C3B006C616E6764721C
:100970006168743B0068696D6D656C3B00617574FE
:100980006F3B0066616872656E3B007472656666F7
:10099000656E3B006B6162656C3B0066696E646509
:1009A0006E3B006B617566656E3B00696E746572C7
:1009B0006E65743B0072656C6169733B006C616EBF
:1009C00067796167693B0064726568656E3B0072B8
:1009D0006F746F723B0067726F756E64706C616EDE
:1009E000653B006B61656C7465723B007765747480
:1009F00065723B00736F6E6E653B00726567656E76
:100A00003B006765736568656E3B006C616E67658A
:100A10003B0074657565723B007072756566756E36
:100A2000673B0073746174696F6E3B0073656E643D
:100A300065723B0079616573753B00656C65637237
:100A40006166743B006B656E776F6F643B00676532
:100A500061726265697465743B00656E6473747578
:100A600066653B006C65696465723B007369636829
:100A700065723B00676562656E3B006D6F7267650E
:100A80006E3B0073757065723B006665726E7365D0
:100A900068656E3B006D6F6E69746F723B00636FCB
:100AA0006D70757465723B00776F7274653B006C96
:100AB00065697374756E673B00626564696E67751E
:100AC0006E673B007363686C656368743B006265C6
:100AD000737365723B00637561676E3B0078637585
:100AE000733B00636F6E64783B00696E666F726D76
:100AF0006174696F6E3B006E756D6D65723B006A67
:100B000065747A743B0074617374653B0074656C42
:100B100065666F6E69653B0074656C6567726166DA
:100B200069653B0073706165743B0066727565684A
:100B30003B007370756C653B006B6F6E64656E7324
:100B400061746F723B0073706572726B726569736A
:100B50003B00666C696567656E3B006C697A656E23
:100B60007A696572743B0070726F626C656D3B00F0
:100B70007472696E6B656E3B00657373656E3B00E6
:100B8000656C6275673B0061776172643B0062650A
:100B900064696E67756E673B00686F6262793B00DF
:100BA000616D617465757266756E6B3B007361741F
:100BB000656C6C69743B006675737362616C6C3B49
:100BC00000747261756D3B006578706572696D6562
:100BD0006E743B00646575746C6963683B00736395
:100BE000687765723B006C65696368743B00756E7D
:100BF0007465723B007374756E64656E3B006D695D
:100C00006E7574656E3B006B6F6D6D656E3B006B52
:100C10006F7066686F657265723B006C61757473A6
:100C2000707265636865723B00696E666F726D69AC
:100C30006572656E3B00647275636B656E3B006D3B
:100C40006F72736574617374653B00636F6E746576
:100C500073743B00686F6262793B00766F726D69F6
:100C600074746167733B006C65697365723B006CFB
:100C700061757465723B00726164696F3B006475F5
:100C80007263683B00676567656E3B006D65746500
:100C9000723B006E6562656C3B00657572656E3B0C
:100CA0000077656E69673B007669656C653B00752A
:100CB0006872656E3B0073746966743B006573739C
:100CC000656E3B00736F6761723B00686562656CBF
:100CD0003B0074617374653B006B657965723B0022
:100CE0006861656E64653B0073656E6465723B00A8
:100CF0006C616D70656E3B0066696C7465723B007B
:100D00007469656665723B00686F656865723B0073
:100D10007765697465723B00736F7267656E3B003F
:100D200064756D6D65723B006172626569743B004C
:100D30007A696568656E3B00736F6E6E69673B002C
:100D4000686F6572656E3B00776F6C6B69673B001F
:100D5000676C656963683B006D75737465723B0011
:100D600066756E6B65723B0068656C6665723B000C
:100D70006272696566653B00626567696E6E3B001D
:100D8000616C6C65696E3B0066657269656E3B00FF
:100D90006C616E6765733B0066696E6465743B00E9
:100DA000676C617562653B006469706C6F6D3B00D8
:100DB000616E7465696C3B006D6F7273656E3B00AC
:100DC0007363686C61663B006B72696567653B00C5
:100DD0006B6F6D6D656E3B00667265756E643B0092
:100DE000686F657265723B006B617374656E3B0082
:100DF00073696562656E3B006272696E67743B0081
:100E00007363686164653B006B6F7374656E3B0070
:100E10006B61727465693B007361756265723B005A
:100E200066696E6765723B00616273696368743BF3
:100E300000747261656765723B0073746F657265FB
:100E40006E3B0067726F657373653B006C6F676222
:100E50007563683B007665726D65726B3B0068690F
:100E60006E776569733B00617262656974653B000A
:100E700066696E646573743B006E6F74697A656E43
:100E80003B0067656C6573656E3B006E6F63686DF4
:100E9000616C3B00766F726C6167653B006C616EE4
:100EA0006773616D3B007363686E656C6C3B007AC1
:100EB00065696368656E3B00676C65696368653B7F
:100EC000006461676567656E3B006672756568659D
:100ED000723B0064617565726E643B0067657261A8
:100EE0006574653B006765686F6572743B0062728C
:100EF00061756368653B006765737465726E3B007E
:100F00007A756B756E66743B006D6574686F6465A9
:100F10003B00617274696B656C3B0067656D616372
:100F200068743B006B6C696E67656C3B0077696346
:100F3000687469673B00736368776163683B00624C
:100F400072696E67656E3B007775657264656E3BAE
:100F5000006265736F7267653B006B6174616C6FF3
:100F6000673B0064756E6B6C65723B006C6165730A
:100F70007469673B007363686E6974743B007370D7
:100F800072616368653B00676564616E6B653B0019
:100F900061757373696368743B0073696E6E766F15
:100FA0006C6C3B0074617374617475723B006E61AC
:100FB00063687465696C3B00646168696E7465722E
:100FC0003B007665726B617566653B0067657769A6
:100FD0006E6E65723B0065726C65646967743B0098
:100FE0006D616E63686D616C3B0062616E64706C14
:100FF000616E3B007363687765737465723B00765E
:1010000065726C696572656E3B007363686E656CD2
:101010006C65723B0061626B7565727A656E3B0050
:10102000616D6174657572656E3B006E6F74697A8F
:10103000627563683B00766F726D65726B656E3BBF
:1010400000626C656973746966743B0067656E6104
:1010500075657265733B006772756E647361747A4F
:101060003B006265686F657264656E3B0067656E24
:101070006175657265733B006D6974686F65726553
:101080006E3B00616C6C67656D65696E3B006E6FF1
:101090007477656E6469673B006E6163687269634B
:1010A00068743B006765627261756368743B006BCE
:1010B00075727A77656C6C653B0062657275666CFB
:1010C0006963683B0077756E6465726261723B00AC
:1010D00064616368626F64656E3B0065696E736529
:1010E000697469673B00766F727A65697469673BFA
:1010F000006765726164656175733B007665726255
:1011000072617563683B00627563687374616265E0
:101110003B006D6568726D616C69673B0062657765
:10112000756E646572743B006861657566696765B4
:10113000723B006C616E646B617274653B00766536
:1011400072736F7267656E3B007765726B73746163
:1011500074743B006265697472616567653B006D1C
:10116000657373706C61747A3B0065696E7370723D
:101170007563683B00656973656E6261686E3B000C
:10118000776F6572746C6963683B006E6163686653
:10119000726167653B0061757373756368656E3B6B
:1011A0000062656D65726B6261723B00756E6265AF
:1011B0006B616E6E743B006E6F6572646C69636820
:1011C0003B00666F65726D6C6963683B00617066B9
:1011D000656C73696E653B00726F73656E62656501
:1011E000743B006D6F65676C696368653B00766F83
:1011F00072736963687469673B0073746F657265C5
:101200006E6465733B006E61656368746C696368E6
:101210003B00766F726D6974746167733B0067722F
:1012200075656E646C6963683B006E6163687465C4
:10123000696C69673B00756E676573746F6572747E
:101240003B0077756E646572766F6C6C3B006672FE
:10125000616E6B72656963683B0065696E73696393
:10126000687469673B007469656673696E6E696767
:101270003B0067726F737361727469673B007669D4
:10128000656C7365697469673B007472616E73693C
:1012900073746F723B006C6F65746B6F6C62656E1C
:1012A0003B006D6573736765726165743B007765BC
:1012B00074746265776572623B00676567656E731B
:1012C000656974653B0073757065726D61726B74EE
:1012D0003B0073746F6572756E67656E3B006C657D
:1012E000697374756E67656E3B00676573756E64D0
:1012F000686569743B00756E7465726B756E6674B3
:101300003B0066756E6B667265756E643B00697353
:101310006F6C61746F72656E3B00766572616272AC
:10132000656465743B00696E666F726D61746976A1
:101330003B00756562657273696368743B00766F24
:1013400072736368726966743B00676C7565636B82
:101350006C6963683B00667265756E646C6963688E
:101360003B006D6974676C69656465723B0061750B
:10137000666D65726B73616D3B0072756E64737040
:10138000727563683B0061626B7565727A756E6732
:101390003B00747265666670756E6B743B007769AE
:1013A0006465727370727563683B006461656D702B
:1013B00066756E673B006162656E6468696D6D6538
:1013C0006C3B00776F6C6B656E6C6F733B00756E7A
:1013D000667265756E646C6963683B007465696C00
:1013E0006E65686D65723B00666C6F686D61726BEF
:1013F000743B0072756E6473747261686C65723BE5
:10140000006665726E737465756572756E673B0014
:1014100061627370616E6E656E3B007565626572C8
:1014200074726167656E3B00646973706C61793BCF
:1014300000736F6E6E656E666C65636B656E3B0008
:101440006D6178696D616C3B00756E676C6175628A
:101450006C6963683B00706C6174696E653B006425
:101460007265686B6F6E64656E7361746F723B005A
:10147000766572626573736572756E673B0062654F
:10148000736368776572656E3B006E616368626165
:10149000727363686166743B00616C7465726E613F
:1014A000746976653B006F737A696C6C61746F72F6
:1014B0003B006261756D61726B743B0062617573B4
:1014C00061747A3B0065696E7374656C6C756E67E8
:1014D0003B00706172616D657465723B00686F639B
:1014E000687061737366696C7465723B00656D69E1
:1014F00074746572736368616C74756E673B0066C3
:10150000656C64656666656B747472616E7369732D
:10151000746F723B00726F746F727374657565726D
:10152000756E673B00736368616C746E65747A7482
:1015300065696C3B00727568657374726F6D3B0012
:101540006C657563687464696F64653B006B617496
:10155000686F64653B006C696368747175656C6C79
:10156000653B007369676E616C3B00736368616C17
:1015700074706C616E3B00706C6174696E656E6C4A
:1015800061796F75743B007A656974756E673B00AD
:10159000717561647261743B00706172616C6C653D
:1015A0006C3B0073657269656C6C3B00756D7363B1
:1015B00068616C7465723B0061757373696368740C
:1015C0003B007669656C6C65696368743B007365A4
:1015D0006C74656E3B0073746164743B0061757478
:1015E0006F6261686E3B007061726B706C61747ADF
:1015F0003B006469676974616C3B006B616D657287
:10160000613B007472616E736365697665723B005D
:101610007261737465723B00616C61726D3B006E48
:101620006F7466616C6C3B00706F6C697A65693BC6
:1016300000756D726563686E656E3B007A657273E6
:10164000746F6572656E3B0062616B656E3B007521
:101650006D7365747A65723B00617573627265695A
:1016600074756E673B006E6577636F6D65723B00E6
:1016700076657273746568656E3B00656D70666152
:101680006E67656E3B0073656E64656E3B007363E9
:10169000686C6166656E3B006E616368743B0061F7
:1016A0007566676577616368743B00776561746828
:1016B00065723B00736F6C61723B00666F726563AD
:1016C0006173743B00736F6C646572696E673B0095
:1016D0006D6F6E69746F72696E673B00696E7472CC
:1016E000756465723B007265706561743B00706F74
:1016F00072746162656C3B0064656E6B6261723B23
:10170000006865726273743B0077696E7465723B42
:1017100000736F6D6D65723B0066727565686C690C
:101720006E673B007363686E65653B006175736649
:101730006C75673B0062616E646272656974653BDB
:1017400000746165676C6963683B007374756465F8
:101750006E74656E3B0073636875656C65723B0003
:101760006C65687265723B006261757374656C6C60
:10177000653B006C6562656E3B0062617573746504
:10178000696E653B00756E76657273636861656D41
:10179000743B00726563686E656E3B006D697473BF
:1017A000636872656962656E3B007A75686F657221
:1017B00065723B006661636867657363686165664F
:1017C000743B0073746174697374696B3B00776573
:1017D00074746572626572696368743B00726567F0
:1017E00069737472696572656E3B007363616E6ED6
:1017F00065723B006E65757765727469673B006260
:101800006C69747A3B0077696E647261643B007541
:10181000726C617562736F72743B006B6F6D706197
:101820006B743B006665726E67657374657565728F
:10183000743B00616C6B6F686F6C3B00766F72730A
:10184000747566653B0034093C0943094A0952092D
:101850005A0963096A0975097D0983098B09940985
:101860009B09A309AB09B509BD09C709CF09D60969
:10187000E309EC09F409FB09020A0B0A120A190A26
:10188000230A2C0A340A3B0A450A4E0A5A0A640AF9
:101890006C0A740A7B0A830A8A0A950A9E0AA80AB5
:1018A000AF0AB90AC40ACE0AD60ADD0AE30AEA0A6E
:1018B000F70AFF0A060B0D0B180B240B2B0B320B30
:1018C000390B460B520B5B0B670B700B790B800BC4
:1018D000870B8E0B990BA00BAD0BB70BC10BC80B75
:1018E000D40BDE0BE60BEE0BF50BFE0B070C0F0C0F
:1018F0001B0C290C360C3F0C4B0C540C5B0C670C6E
:101900006F0C770C7E0C850C8C0C930C9A0CA10C34
:10191000A80CAF0CB60CBD0CC40CCB0CD20CD90C63
:10192000E00CE80CF00CF80C000D080D100D180D73
:10193000200D280D300D380D400D480D500D580D5F
:10194000600D680D700D780D800D880D900D980D4F
:10195000A00DA80DB00DB80DC00DC80DD00DD80D3F
:10196000E00DE80DF00DF80D000E080E100E180E2B
:10197000200E280E310E3A0E430E4C0E550E5E0E02
:10198000670E700E790E820E8B0E940E9D0EA60EB3
:10199000AF0EB80EC10ECA0ED30EDC0EE50EEE0E63
:1019A000F70E000F090F120F1B0F240F2D0F360F0C
:1019B0003F0F480F510F5A0F630F6C0F750F7E0FBB
:1019C000870F900F9A0FA40FAE0FB80FC20FCC0F56
:1019D000D60FE00FEA0FF40FFF0F0A1015102010BA
:1019E0002B10361041104C10571062106D107810EB
:1019F00083108E109910A410AF10BA10C510D0101B
:101A0000DB10E610F110FC10071112111D11281146
:101A100033113E11491154115F116A117511801172
:101A20008B119611A111AC11B711C211CD11D811A2
:101A3000E311EE11FA11061212121E122A123612B8
:101A400042124E125A12661272127E128A129612A6
:101A5000A212AE12BA12C612D212DE12EA12F61296
:101A600002130E131A13261332133E134A1356137E
:101A700062136E137A13861392139E13AB13B6136D
:101A8000C313CE13DC13E813F313011410141B1447
:101A9000281431144014491456145F1470147E1421
:101AA0008A149914A614B214BC14C514D214DD14EB
:101AB000ED14FF1415152515351540154D15561542
:101AC00063156B157715871590159915A315AC152A
:101AD000B815C215CE15D615DD15E715F215FB158F
:101AE0000316101618161F16281631163C1648161F
:101AF0004F165916661670167B1686168E16981691
:101B00009F161E12B416BB16C516D016DC16E616A6
:101B1000EE16F816011709171117191724172C17A5
:101B2000351741174B1756176017681773177A1731
:101B3000851793179C17AA17B417C317CE17DD176D
:101B4000EB17F417FF1706180F181B182418331873
:101B50003C18646C386B666F20646520646C316B74
:101B60006270203D20746E782066657220727072FB
:101B700074203539392066726F6D20636F6C6F6722
:101B80006E65203D20757220727374206973203554
:101B900037392035376E203D2071746820697320F5
:101BA0006E722061616368656E2061616368656E55
:101BB000203D206E616D65206973206672616E6BD9
:101BC000206672616E6B203D20687065206F6B3FF0
:101BD00020646C386B666F20646520646C316B62C6
:101BE0007020707365206B3B0077387973642064D4
:101BF0006520646C3274756E203D20616C6C2072BF
:101C000069676874206465617220627279616E2010
:101C10003D2071736C207669612062757265617513
:101C2000206F6B203D20746E7820666572206E698F
:101C300063652071736F20616E642061206E69633B
:101C400065207765656B656E64203D206870652052
:101C5000637561676E20736F6F6E203D20773879F2
:101C6000736420646520646C3274756E206E772016
:101C7000717274206520653B00646C366B626C2069
:101C800064652069356F7066203D206578637573E3
:101C9000206472206F6D2062656E203D2068722086
:101CA0006E696C20696E666F20616274206D7920A8
:101CB0006F75747074203D206D7920707772206D7F
:101CC0007472206E696C206F6B203D2070612074EF
:101CD000627320327836313436203D20696E70745C
:101CE00020616274203136302077747473203D2077
:101CF000646C366B626C2064652069356F70662099
:101D0000707365206B3B00646A316B6B6F20646598
:101D1000206561396D63203D20616C6C206F6B2004
:101D2000647220616C62657274203D20707365205E
:101D3000717270203D207572207369676E2076790C
:101D4000206764203D2072737420356E6E20356EDE
:101D50006E203D206D79207478206F75747074202A
:101D60006E7720322077747473203D20687720636B
:101D700070693F203D20646A316B6B6F2064652081
:101D80006561396D6320707365206B3B00646C3452
:101D90006661206465206862396C71203D206F6B3C
:101DA000206D79207369677320727374203436391B
:101DB00020736F2061676E206D6E6920746E7820CD
:101DC00066657220696E666F203D206D7920616EB8
:101DD0007420666572203430206D74727320322056
:101DE000656C207961676920736F20737572652057
:101DF000776C2063706920796F7520746D77206F20
:101E00006E2037303032206B687A203D20646C348D
:101E10006661206465206862396C7120707365208A
:101E20006B3B00646B396172206465206467386BBA
:101E30006372203D20746E78206665722063616C49
:101E40006C20647220667264203D20757220736974
:101E5000676E20727374203337386B203337386BDA
:101E60003D20717468206B617373656C206573200D
:101E70006E616D652077696C6C69203D20726967C1
:101E800020747276637220686F6D656D6164652081
:101E900066657220637720657320737362203D202E
:101EA00070777220616274203520777474732061BA
:101EB0006E74206469706F6C65203D2068772063C4
:101EC00070693F203D20646B396172206465206435
:101ED00067386B637220707365206B3B00646637F4
:101EE0006F6C78206465207061336572203D2076C8
:101EF0007920737269206472206F6D206B6C61753C
:101F000073203D206E696C206370692075722073A8
:101F1000696773203D2061676320696E206D7920B9
:101F20007472637672206E696C206F6B203D207036
:101F300073652035206D696E203D20776C206361CC
:101F40006C6C20752061676E20736E203D20616788
:101F50006E206578637573203D206466376F6C78FA
:101F60002064652070613365723B00646C3976676C
:101F700020646520646A33776173203D206775743F
:101F8000656E206162656E64206C696562657220B1
:101F9000746F6E69203D207363686F656E2064699D
:101FA0006368207A7520686F6572656E203D2064D5
:101FB00065696E2072737420697374203539392015
:101FC000356E6E203D2069636820686F6666652CFB
:101FD00020647520686174746573742065696E652A
:101FE0006E20677574656E207461673F203D2064C4
:101FF0006C39766720646520646A3377617320707A
:102000007365206B3B00646B3478792064652064D1
:102010006C376B7A6F203D206E65696E2C206D6980
:10202000636861656C206963682068616265206B24
:1020300065696E65206E65756520616E74656E6E8E
:1020400065203D20616E7420666233332066623302
:1020500033203D20667565722032306D20726569CF
:10206000636874206D69722064617320766F6C6C94
:102070006B6F6D6D656E206869203D2077616E6EB7
:10208000206B6F6D6D742064656E6E206465696E83
:10209000206E65756572206D6173743F203D20640C
:1020A0006B34787920646520646C376B7A6F2070AC
:1020B0007365206B3B007731617720646520646C29
:1020C000397A6D203D2073746E2068722037357424
:1020D0002077747473206F75747075742065732025
:1020E000616E74203520656C2079616769206162BA
:1020F00074203138206D7472207570203D207778FF
:1021000020756662207769642074656D70203330B5
:102110002063203D20707365207173792032206B1D
:10212000687A2064776E203D2068722071726D207D
:1021300066726D20727474792073746E203D207005
:102140007365206B3B006466346B782064652064A3
:102150006A316A77203D20676D206C627220756C51
:102160006C6920657320766C6E20646B20666572E6
:1021700020696E666F2061627420636F6E74657390
:1021800074203D20636F6E647320756662203D206D
:1021900070736520717271203D206D7920727820F6
:1021A000686F6D656D6164652077696420323320E6
:1021B000746273203D20777820666220323120637C
:1021C000203D20687065206177646820746D7720F9
:1021D0003D3D3B00646D39656520646520646B3866
:1021E0007A66203D206861626520686965722073A7
:1021F0007461726B65732071726D206475726368AF
:102200002065696E652073746174696F6E206175F5
:102210007320796F203D20696872206E616D6520A2
:10222000756E64206968722071746820776172200D
:102230006E69636874206175667A756E65686D6530
:102240006E203D20626974746520676568656E2044
:10225000736965207A756D2073656E64656E2035CF
:10226000206B687A20686F65686572203D206D6517
:10227000696E206E616D6520697374206B61726C8C
:102280006865696E7A20756E64206D65696E20716F
:102290007468206973742077616C6473617373650B
:1022A0006E206E72206F6B206772656E7A65203DBE
:1022B0003B007761327177206465206F6E35666B05
:1022C000203D206765206472206F6D20626F622060
:1022D0006573206D6E6920746E7820666572207556
:1022E00066622072707274203D2075722073696777
:1022F00073206872206E772072737420343739200F
:1023000034376E203D206D792073746E20747263B3
:1023100076722077696420313030207720696E70C2
:102320007420657320616E74206770203D20707387
:1023300065206B3B006B31777320646520646C32E1
:10234000777973203D206F6B2077696420696E6612
:102350006F20616274207572207269672064722038
:102360006F6D206A696D203D20687220726376640B
:1023700020616C6C206662203D2068772061627469
:1023800020736B65642066657220746D77206F6EB4
:102390002031306D203F203D2071727620696E2003
:1023A00073737476203D2071726B3F203D206B313A
:1023B000777320646520646C32777973207073655D
:1023C000206B3B006B613161626320646520707932
:1023D000306D6167203D20756662206472206672F0
:1023E00064203D207073652075722071736C2077B6
:1023F00069642073616520657320322069726320EF
:102400003D20776C2071736C20766961206469725D
:1024100065637420657320737572652063666D2033
:1024200073776C207270727473203D3D3B0066338D
:10243000747220646520646A39707771203D20755C
:102440007220727072742072737420353939203D95
:102450002073756D20717362203D20707772206843
:102460007220373520777474732066726D20686F20
:102470006D656D616465207478203D20676C207700
:102480006964207572206177617264203D206D6EF1
:10249000692073746E732066726D20646C20776C93
:1024A0002063616C6C20696E207465737420746D98
:1024B00077203D3D3B00646A316A77206465206483
:1024C0006C326B7467203D206761206C6272206FF4
:1024D0006D2073746566616E20657320746E78205C
:1024E0006665722063616C6C203D2075722072738A
:1024F000742069732035393920356E6E206573205C
:102500007566622073696773203D206D7920717450
:1025100068206973207374757474676172742073B2
:102520007475747467617274203D206E616D6520EE
:10253000616E647265617320616E6472656173209F
:102540003D20687065206F6B3F20646A316A772098
:10255000646520646C316B746720707365206B3B1D
:1025600000646B316F7420646520646D347A746626
:10257000203D2068616C6C6F206C6965626572201B
:1025800072616C66203D207363686F656E2C206DF0
:10259000616C2077696564657220766F6E2064696E
:1025A00072207A7520686F6572656E203D206973B0
:1025B0007420616C6C6573206F6B61792062656952
:1025C00020657563683F20776173206D616368746F
:1025D000206469652078796C3F2077697220747275
:1025E000656666656E20756E73206E6165636873DF
:1025F000746520776F636865207A756D2066642C3A
:10260000206B6F6D6D742069687220617563683F1F
:1026100020646B316F6220646520646D347A746667
:1026200020707365206B3B006737756E20646520F2
:10263000646C33727462203D206765206472206F81
:102640007020657820746E7820666572207572201F
:102650007270727420353939203D20757220727382
:10266000742069732035393920356E6E20746F6F90
:10267000203D20796F7572206B3320697320756659
:1026800062203D206D79207269672069732069633B
:102690006F6D20373630302069636F6D20373630EC
:1026A00030207077722031747420777474732061D5
:1026B0006E74203320656C206265616D203D207151
:1026C0007468206D756E696368206D756E696368E6
:1026D000203D206737756E20646520646C3372740A
:1026E0006220707365206B3B00646A366B626C20FD
:1026F000646520646C387A706C203D2068616C6C75
:102700006F206469657465722C207669656C656EEE
:102710002064616E6B2066756572206465696E6504
:102720006E207270727420353739203D206D6569D6
:102730006E20756D7A756720696E73206E6575659C
:10274000207174682069737420696E203220776F5D
:102750006368656E203D2069636820686F66666502
:102760002C206461737320646572206D6173742022
:102770006E616563687374657320776F6368656EF7
:10278000656E646520617566676562617574207742
:10279000697264203D20373320756E64206269734E
:1027A000207A756D206E616563687374656E206F45
:1027B00076206162656E64203D20646A366B626CCF
:1027C00020646520646C387A706C20707365206BAF
:1027D0003B006467367472206465206C61316173FC
:1027E000203D20746E7820666572207270727420AD
:1027F000647220616E6472656173203D206D792082
:102800007269672069732061206B656E776F6F64F2
:10281000207473353930207473353930203D207081
:102820007772206E7720353020777474732035747A
:102830002077747473203D20616E74206973206763
:102840003572762067357276203D20777820657264
:102850006520697320736E6F772061627420312068
:1028600063203D206D6E6920746E7820666572204D
:1028700071736F203D2071736C206F6B20766961DE
:1028800020627572656175203D20707365206B3B19
:1028900000646C3161626320646520646B356C7424
:1028A00072203D206761206C6272206F6D206A6F1C
:1028B000616368696D203D206861626520766F6E96
:1028C000206465696E656D206572666F6C67206255
:1028D00065696D206B6F6E74657374206765686FD2
:1028E0006572742C20636F6E6772617473203D2073
:1028F00062697374206475206E61656368737465C2
:1029000020776F636865206175662064656D206659
:1029100069656C6464617920766F6D206F762064E0
:10292000616265693F2069636820777565657264D7
:1029300065206D6963682066726575656E203D3D32
:102940003B006466376B627620646520646C386691
:102950007767203D20737269206C6272206F6D2052
:102960006672616E7A203D20727374203332392092
:10297000333239203D2064657220737475726D2086
:102980006C65747A746520776F636865206861741C
:10299000206D65696E6520616E74656E6E6520627E
:1029A00065736368616564696774203D20696D20A3
:1029B0006D6F6D656E74206B616E6E20696368204B
:1029C0006E7572206D6974206469706F6C20756E0D
:1029D0006420313020777474732073656E64656E83
:1029E000203D20686F6666652C206475206B616EE3
:1029F0006E7374206D69636820656D7066616E67C3
:102A0000656E3F20707365206B3B00646C396464B5
:102A100071206465207061317771203D20676520E9
:102A20006472206F6D2074686F6D61732065732010
:102A3000746E78206665722063616C6C203D206442
:102A400065696E20727374206973203539392035B9
:102A50007474203D20717468206973206E65617202
:102A600020726F65726D6F6E6420726F65726D6F2C
:102A70006E64203D206E616D652069732070686909
:102A80006C207068696C203D207269672069732032
:102A90007961657375206674323030302066743227
:102AA00030303020707772206E7720383020777485
:102AB0007473203D206F6B3F20646C396464712017
:102AC000646520706131777120707365206B3B0005
:102AD000646C326B626420646520646A336B6B7073
:102AE000203D206E65696E206265726E642C2064E4
:102AF00075206769627374206E6F636820696D6DFD
:102B0000657220736F207363686C656368742077E7
:102B100069652064616D616C73203D207669656C28
:102B20006C65696368742077616572652073736290
:102B300020656865722065747761732066756572BB
:102B400020646963683F206869203D20646C326BB3
:102B5000626420646520646A336B6B7020707365F7
:102B6000206B3B00646C3369666120646520646B94
:102B70003976667A203D206774206F6D206D617212
:102B800074696E203D20646B2066657220727566E4
:102B9000203D2075722035393920356E6E20696EE2
:102BA000206B656C6B6865696D206B656C6B686527
:102BB000696D203D20646F6B2066323720663237A6
:102BC000203D206E616D6520776F6C6667616E6772
:102BD00020776F6C6667616E67203D2064652064B6
:102BE0006B3976667A20707365206B3B00646130C8
:102BF0006161206465206462397A7A203D207566BF
:102C00006220647220667264203D207073652075B6
:102C1000722071736C20776964207361652065731D
:102C2000203220697263207669612064697265636D
:102C30007420657320737572652063666D207377E9
:102C40006C207270727473203D20746E78206665FB
:102C5000722071736F2065732068706520637561E1
:102C6000676E20736E203D20646130616120646571
:102C7000206462397A7A20707365206B3B00646748
:102C8000386B637220646520646D316F676B203D23
:102C9000206E65696E206C6272206A616E206963C5
:102CA000682068616265206E6F6368206E69636882
:102CB000747320766F6E206465696E656D206E6535
:102CC00075656E20717468206765736568656E2030
:102CD0003D2073746568742064656E6E2064656958
:102CE0006E6520616E74656E6E65207363686F6ECD
:102CF0003F2064616E6E206B6F6D6D652069636847
:102D0000206D6F7267656E206D616C20766F7262E8
:102D10006569203D206467386B63722064652064B8
:102D20006D316F676B20707365206B3B00646C3294
:102D3000616C6120646520646B37766A76203D2083
:102D400070736520717270203D2077697220776FF3
:102D5000686E656E203130206B6D20656E7466651F
:102D6000726E742C20646120627261756368737482
:102D7000206475206B65696E652037353020777467
:102D80007473203D20696368206B616E6E206469F6
:102D90006368206C61757420756E64206465757459
:102DA0006C69636820686F6572656E203D20646C95
:102DB00032616C6120646520646B377676207073B5
:102DC00065206B3B00646C396B6B75206465206417
:102DD0006C35746577203D2068616C6C6F206C6287
:102DE000722072616C66203D206861737420647586
:102DF000206465696E656E206B3220656E646C6957
:102E00006368206665727469673F206B6C696E67E2
:102E10007420677574203D20727374203537392013
:102E200035376E203D206D65696E6520616E746575
:102E30006E6E65206973742065696E203420656C40
:102E4000206265616D203D20707772206162742080
:102E50003230302077747473203D20616C6C206FA9
:102E60006B3F20707365206B203D3D3B00521BE99A
:102E70001B791C071D8D1D231EDD1E6B1F0620B632
:102E8000204621D421B2223523C4232E24B6246126
:102E9000252826E926D227912842290B2AD02A6400
:102EA0002BED2B7E2C2D2DC52D000000002400279E
:102EB000002A0000000000250028002B0000000070
:102EC000002300260029000404040404040404026E
:102ED00002020202020303030303030102040810B7
:102EE0002040800102040810200102040810200084
:102EF00000000700020100000304060000000000BB
:102F00000000000216183F3411241FBECFEFD8E096
:102F1000DEBFCDBF15E0A0E0B1E0E4E9F2E702C01A
:102F200005900D92A031B107D9F716E0A0E1B5E008
:102F300001C01D92AE30B107E1F71FE2C8E0DFE249
:102F400004C02297FE010E940D39C430D107C9F791
:102F50000E948F340C9448390C940000A0E0B0E03B
:102F6000E4EBF7E10C941939EC01A880B980CA8030
:102F7000DB80A114B104C104D10441F484E2A82E81
:102F800089EDB82E8BE5C82E87E0D82EC601B50195
:102F90002DE133EF41E050E00E94DC3827EA31E4D4
:102FA00040E050E00E9488387B018C01C601B501E9
:102FB0002DE133EF41E050E00E94DC38CA01B90155
:102FC0002CEE34EF4FEF5FEF0E9488386E0D7F1DBF
:102FD000801F911F97FF04C061507040804090484F
:102FE000688379838A839B839B01AC015F77B901F6
:102FF000CA01CDB7DEB7EAE00C9435390E94AE17AE
:1030000008958EE293E00E94AE17089560932E0318
:1030100070932F0380933003909331030895FB0145
:10302000DC0105900D920020E1F70895CF92EF9218
:103030000F9380E195E06CE04BE025E004E073E065
:10304000E72E52E0C52E0E945F302091340330916C
:1030500035033093260520932505C901880F991F54
:10306000820F931F90932805809327050F91EF906F
:10307000CF900895CF93DF938091290590912A05F1
:10308000892BA9F0C0E0D0E00BC0609125057091BC
:103090002605882777FD8095982F0E94F33021968A
:1030A0008091290590912A05C817D90774F360917A
:1030B000250570912605660F771F882777FD809577
:1030C000982F0E94F330DF91CF91089560913603DD
:1030D000709137038091320320E030E040E050E00F
:1030E0000E942A366091270570912805882777FD70
:1030F0008095982F0E94F330809132030E94B7355B
:103100006091250570912605882777FD8095982F79
:103110000E94F330089560913603709137038091D7
:10312000320320E030E040E050E00E942A36609117
:10313000250570912605882777FD8095982F0E9498
:10314000F330809132030E94B7356091250570916C
:103150002605882777FD8095982F0E94F3300895E3
:10316000809132036CED75E020E030E040E050E00B
:103170000E942A3662E370E080E090E00E94F33023
:10318000809132030E94B73508951F93182F6091E4
:103190004505709146056F5F7F4F709346056093BC
:1031A000450580E195E041E00E94722F8091450540
:1031B000909146054097B4F080E195E060E041E0F1
:1031C0000E94722F80E195E060E071E00E949335EB
:1031D00080E195E060E041E00E94722F1092460588
:1031E0001092450580E195E0612F0E945E2F1F91AE
:1031F00008952091250530912605B901660F771FA6
:10320000620F731F660F771F882777FD8095982FB1
:103210000E94F33080E20E94C5180895992787FD27
:103220009095A92FB92FFC01B097EB35F10508F067
:10323000F0C1EC5CFF4FEE0FFF1F0590F491E02D05
:1032400009940E948B180E9466180E943A1881E423
:10325000DBC10E9466180E948B180E948B180E9486
:103260008B180E943A1882E4CFC10E9466180E940F
:103270008B180E9466180E948B180E943A1883E4EB
:10328000C3C10E9466180E948B180E948B180E946E
:103290003A1884E4B9C10E948B180E943A1885E458
:1032A000B3C10E948B180E948B180E9466180E945E
:1032B0008B180E943A1886E4A7C10E9466180E94E3
:1032C00066180E948B180E943A1887E49DC10E94DC
:1032D0008B180E948B180E948B180E948B180E94DA
:1032E0003A1888E491C10E948B180E948B180E94A2
:1032F0003A1889E489C10E948B180E9466180E94BE
:1033000066180E9466180E943A188AE47DC10E94DD
:1033100066180E948B180E9466180E943A188BE467
:1033200073C10E948B180E9466180E948B180E941D
:103330008B180E943A188CE467C10E9466180E949C
:1033400066180E943A188DE45FC10E9466180E94B8
:103350008B180E943A188EE457C10E9466180E948A
:1033600066180E9466180E943A188FE44DC10E94A8
:103370008B180E9466180E9466180E948B180E9483
:103380003A1880E541C10E9466180E9466180E94A2
:103390008B180E9466180E943A1881E535C10E9478
:1033A0008B180E9466180E948B180E943A1882E5BA
:1033B0002BC10E948B180E948B180E948B180E94B0
:1033C0003A1883E521C10E9466180E943A1884E5E4
:1033D0001BC10E948B180E948B180E9466180E94C5
:1033E0003A1885E511C10E948B180E948B180E9423
:1033F0008B180E9466180E943A1886E505C10E9443
:103400008B180E9466180E9466180E943A1887E579
:10341000FBC00E9466180E948B180E948B180E94A5
:1034200066180E943A1888E5EFC00E9466180E944C
:103430008B180E9466180E9466180E943A1889E547
:10344000E3C00E9466180E9466180E948B180E94B2
:103450008B180E943A188AE5D7C00E948B180E94E8
:1034600066180E9466180E9466180E9466180E94DC
:103470003A1881E3C9C00E948B180E948B180E94E1
:1034800066180E9466180E9466180E943A1882E325
:10349000BBC00E948B180E948B180E948B180E9440
:1034A00066180E9466180E943A1883E3ADC00E9415
:1034B0008B180E948B180E948B180E948B180E94F8
:1034C00066180E943A1884E39FC00E948B180E94DD
:1034D0008B180E948B180E948B180E948B180E94D8
:1034E0003A1885E391C00E9466180E948B180E94CA
:1034F0008B180E948B180E948B180E943A1886E342
:1035000083C00E9466180E9466180E948B180E9451
:103510008B180E948B180E943A1887E375C00E948E
:1035200066180E9466180E9466180E948B180E94F6
:103530008B180E943A1888E367C00E9466180E94A0
:1035400066180E9466180E9466180E948B180E94D6
:103550003A1889E359C00E9466180E9466180E94B2
:1035600066180E9466180E9466180E943A1880E346
:103570004BC00E9466180E9466180E948B180E9419
:103580008B180E9466180E9466180E943A188EE2F4
:103590003BC00E9466180E948B180E948B180E94E4
:1035A0008B180E9466180E943A188DE32DC00E9465
:1035B00066180E948B180E948B180E9466180E9441
:1035C0008B180E943A188FE21FC00E948B180E942D
:1035D0008B180E9466180E9466180E948B180E9421
:1035E0008B180E943A188FE30FC00E9466180E9441
:1035F00066180E948B180E948B180E9466180E9401
:1036000066180E943A188CE20E94C51808950E941C
:10361000F9180895CF92DF92FF920F931F93CF93E3
:10362000DF936C0100E010E02FC080913C0390918B
:103630003D03019749F461E670E080E090E025E801
:1036400030E040E050E008C061E670E080E090E0EB
:103650002BE730E040E050E00E9462386B377105A4
:1036600014F06B547040F62EC0E0D0E004C08F2DF3
:103670000E940E19219680913E0390913F03C81736
:10368000D907ACF30F5F1F4F0C151D0574F20E9494
:10369000F9180E94F918DF91CF911F910F91FF90B7
:1036A000DF90CF900895BF92CF92DF92EF92FF927A
:1036B0000F931F93CF93DF936C01EE24FF24BBE3A2
:1036C000BB2E37C080913C0390913D03019749F494
:1036D00061E670E080E090E025E830E040E050E016
:1036E00008C061E670E080E090E02BE730E040E069
:1036F00050E00E94623868836B3771051CF06B5490
:1037000070406883862F0E940E190F5F1F4F21960D
:10371000E0913E03F0913F030E171F079CF2E65C19
:10372000FA4FB0820E94F9180E94F9180894E11C1F
:10373000F11CEC14FD042CF4CAE3D5E000E010E029
:10374000E7CFDF91CF911F910F91FF90EF90DF9026
:10375000CF90BF900895AF92BF92CF92DF92EF9239
:10376000FF920F931F93CF93DF935C0161E070E0B2
:1037700080E090E02DE330E040E050E00E946238CD
:10378000EB01CC0FDD1FCC0FDD1FC60FD71FCA5BAF
:10379000DC4FEE24FF2488818B3371F00E940E19D8
:1037A000F501EE0DFF1D899180830894E11CF11C49
:1037B00085E0E816F10479F760E370E080E090E0DE
:1037C0002AE330E040E050E00E946238162F862F56
:1037D0000E940E19E501CE0DDF1D188361E670E031
:1037E00080E090E02BE730E040E050E00E9462385B
:1037F000162F862F0E940E19198361E670E080E073
:1038000090E02BE730E040E050E00E946238162F55
:10381000862F0E940E191A83E3E0F0E0EE0EFF1EE1
:103820006501CE0CDF1C8DEF9FEFE80EF91E0BE358
:10383000F601008360E070E080E090E022E030E09C
:1038400040E050E00E9462386130710581059105C9
:10385000A1F461E670E080E090E02BE730E040E02A
:1038600050E00E946238162F862F0E940E19F60132
:1038700010830C830894E11CF11C61E070E080E08F
:1038800090E029E030E040E050E00E94623865308E
:1038900071058105910589F48FE20E940E19850159
:1038A0000E0D1F1D8FE2F801838380E70E940E1921
:1038B00080E7F80184838BE385830E94F918DF9108
:1038C000CF911F910F91FF90EF90DF90CF90BF901D
:1038D000AF9008950F931F93CF93DF938C01C0E0B7
:1038E000D0E0F801EC0FFD1F80818B3339F480911B
:1038F0004405882351F40E94F91807C00E940E194C
:10390000219681E0C030D80761F7DF91CF911F91F8
:103910000F910895CF92DF92EF92FF920F931F9332
:10392000CF93DF936B0121E020934405C0E0D0E00A
:1039300001967C010027F7FC0095102F24C060E061
:1039400070E080E090E0A80197010E9462389B013E
:10395000220F331F260F371FC9018E589B4F0E941D
:103960006A1C61E070E080E090E026E030E040E03A
:1039700050E00E946238643071058105910511F4B0
:103980000E94F9182196CC15DD05CCF21092440561
:10399000DF91CF911F910F91FF90EF90DF90CF902B
:1039A00008950F931F93DF93CF93CDB7DEB7C05029
:1039B000D1400FB6F894DEBF0FBECDBFFC01EE0FB5
:1039C000FF1FE359F14D659174918E010F5F1F4FF9
:1039D000C8010E940F18C8010E946A1C0E94F918B1
:1039E000C050DF4F0FB6F894DEBF0FBECDBFCF91F2
:1039F000DF911F910F9108950F931F93DF93CF9342
:103A0000CDB7DEB76E970FB6F894DEBF0FBECDBF51
:103A1000FC01EE0FFF1FEA5BF74E659174918E017A
:103A20000F5F1F4FC8010E940F18C8010E946A1C37
:103A30000E94F9186E960FB6F894DEBF0FBECDBF88
:103A4000CF91DF911F910F9108950F931F93DF93F3
:103A5000CF93CDB7DEB727970FB6F894DEBF0FBE72
:103A6000CDBFFC01EE0FFF1FE85AF74F659174912F
:103A70008E010F5F1F4FC8010E940F18C8010E94DE
:103A80006A1C0E94F91827960FB6F894DEBF0FBE85
:103A9000CDBFCF91DF911F910F9108950F931F9389
:103AA000DF93CF9300D000D000D0CDB7DEB7FC01BC
:103AB000EE0FFF1FE851FB4F659174918E010F5F70
:103AC0001F4FC8010E940F18C8010E946A1C0E9463
:103AD000F91826960FB6F894DEBF0FBECDBFCF9172
:103AE000DF911F910F9108950F931F93DF93CF9351
:103AF00000D000D00F92CDB7DEB7FC01EE0FFF1F54
:103B0000EA5CFD4F659174918E010F5F1F4FC801F4
:103B10000E940F18C8010E946A1C0E94F9180F9099
:103B20000F900F900F900F90CF91DF911F910F91F9
:103B30000895DF92EF92FF920F931F938C0168E438
:103B4000E62E65E0F62EC701B8010E949830D82E07
:103B50000F5F1F4FC701B8010E949830382F20E037
:103B60002D0D311DC9011F910F91FF90EF90DF9036
:103B7000089580E090E00E94991D9093390380930E
:103B8000380382E090E00E94991D90933703809360
:103B9000360384E090E00E94991D90933B0380934C
:103BA0003A0386E090E00E94991D90932A05809345
:103BB000290588E090E00E94991D9093410380932D
:103BC00040038AE090E00E94991D90933303809314
:103BD00032038CE090E00E94991D90932C05809315
:103BE0002B058EE090E00E94991D90933D038093F9
:103BF0003C0380E190E00E94991D909339058093E9
:103C0000380582E190E00E94991D90933F038093D4
:103C10003E0308950F931F930E94B91D80913203B4
:103C200061E00E94B33186E060E00E94B33186E03B
:103C300061E00E94D93188E060E00E94B33188E001
:103C400061E00E94D93187E060E00E94B33187E0F3
:103C500061E00E94D9318AED95E040E855E260E0EC
:103C600070E00E94113380E00E9491310E94803800
:103C700000E115E0C80160E142E020E00E94A92FC8
:103C8000C80161E171E00E949335C8016DE171E006
:103C90000E949335C80160E041E00E94722FC80184
:103CA00063E271E00E94933564EC79E080E090E09B
:103CB0000E94F330C8010E94A12F609138037091D7
:103CC000390380EB94E00E94A738CB017093350351
:103CD0006093340370932605609325059B01220FA2
:103CE000331F280F391F30932805209327051F9174
:103CF0000F910895DF92EF92FF920F931F938C0123
:103D0000462FD72EE8E4EE2EE5E0FE2EC701B801DF
:103D10000E949F300F5F1F4FC701B8014D2D0E94B9
:103D20009F301F910F91FF90EF90DF9008950F93B8
:103D30001F93CF93DF9380E195E00E94A12F80E154
:103D400095E060E040E00E94722F80E195E065E33D
:103D500071E00E94933586E00E942D32892BC9F4D0
:103D6000809144039091450301969093450380937D
:103D700044030A9744F081E090E0909345038093D8
:103D800044030E94B01868EC70E080E090E00E946C
:103D9000F33088E00E942D32892BC1F480914403D6
:103DA000909145030197909345038093440318161F
:103DB000190634F089E090E0909345038093440322
:103DC00068EC70E080E090E00E94F33087E00E94B1
:103DD0002D32892B11F010E007C068EC70E080E014
:103DE00090E00E94F33011E08091440390914503EC
:103DF0008530910509F49AC3863091059CF4823090
:103E0000910509F413C18330910524F4019709F059
:103E100004C718C08330910509F4DEC1049709F086
:103E2000FCC6B1C28730910509F4AFC48730910553
:103E30000CF41CC48830910509F436C5099709F0C3
:103E4000ECC605C680E195E060E041E00E94722F7B
:103E500080E195E06CE371E00E949335113009F048
:103E6000BFC080E195E00E94A12F80E195E060E075
:103E700040E00E94722F80E195E06CE371E00E94C7
:103E8000933580E195E060E041E00E94722F80E18F
:103E900095E06CE471E00E94933580E195E06CE080
:103EA00041E00E94722F609138037091390380E1E4
:103EB00095E04AE050E00E94803566E970E080E0DD
:103EC00090E00E94F330CCE3D0E086E00E942D32F7
:103ED000892B79F58091380390913903019690935D
:103EE00039038093380368EC70E080E090E00E9432
:103EF000F3308091380390913903CD9724F0D0931B
:103F00003903C093380380E195E069E571E00E94D0
:103F1000933580E195E06CE041E00E94722F609162
:103F200038037091390380E195E04AE050E00E9447
:103F3000803588E00E942D32892B89F580913803E5
:103F4000909139030197909339038093380368EC7B
:103F500070E080E090E00E94F3308091380390910F
:103F600039030A9734F48AE090E090933903809300
:103F7000380380E195E069E571E00E94933580E1C6
:103F800095E06CE041E00E94722F609138037091DF
:103F9000390380E195E04AE050E00E94803587E0F7
:103FA0000E942D32892B09F090CF80E195E060E0EE
:103FB00041E00E94722F80E195E060E071E00E9494
:103FC000933580E195E060E041E00E94722F64E665
:103FD00070E080E090E00E94F33081E0809347053C
:103FE0001092460510924505E0913803F09139038F
:103FF00080EB94E0BF010E94A73860933403709374
:104000003503609325057093260520913403309184
:104010003503C901880F991F820F931F90932805BC
:104020008093270580E090E0BF01F5C580E195E031
:1040300060E041E00E94722F80E195E06CE571E064
:104040000E949335112309F4C0C080E195E00E94DD
:10405000A12F80E195E060E040E00E94722F80E1B6
:1040600095E06CE571E00E94933580E195E060E0B9
:1040700041E00E94722F80E195E068E671E00E94C5
:10408000933580E195E06AE041E00E94722F6091F3
:104090003A0370913B0380E195E04AE050E00E94D2
:1040A000803566E970E080E090E00E94F33004EF34
:1040B00011E0C9E1D0E086E00E942D32892B81F524
:1040C00080913A0390913B03499690933B038093F0
:1040D0003A0368EC70E080E090E00E94F330809159
:1040E0003A0390913B03855F914024F010933B038A
:1040F00000933A0380E195E069E571E00E94933511
:1041000080E195E06AE041E00E94722F60913A03FD
:1041100070913B0380E195E04AE050E00E948035D9
:1041200088E00E942D32892B79F580913A03909195
:104130003B03499790933B0380933A0368EC70E00C
:1041400080E090E00E94F33080913A0390913B032D
:10415000499724F4D0933B03C0933A0380E195E060
:1041600069E571E00E94933580E195E06AE041E005
:104170000E94722F60913A0370913B0380E195E0B9
:104180004AE050E00E94803587E00E942D32892B62
:1041900009F091CF80E195E060E041E00E94722F4C
:1041A00080E195E060E071E00E94933580E195E068
:1041B00060E041E00E94722F64E670E080E090E0F1
:1041C0000E94F33081E08093470560913A0370913B
:1041D0003B0384E090E01FC580E195E060E041E0B2
:1041E0000E94722F80E195E062E771E00E949335B2
:1041F000112309F4C1C080E195E00E94A12F80E164
:1042000095E060E040E00E94722F80E195E06BE76E
:1042100071E00E94933580E195E060E041E00E940A
:10422000722F80E195E069E871E00E94933580E1AA
:1042300095E06AE041E00E94722F60913603709130
:10424000370380E195E04AE050E00E94803566E95E
:1042500070E080E090E00E94F33000EB14E0C4EFE7
:10426000D1E086E00E942D32892B81F580913603C2
:1042700090913703C296909337038093360368EC8E
:1042800070E080E090E00E94F330809136039091DE
:104290003703815B944024F0109337030093360377
:1042A00080E195E069E571E00E94933580E195E059
:1042B0006AE041E00E94722F6091360370913703EB
:1042C00080E195E04AE050E00E94803588E00E945D
:1042D0002D32892B81F58091360390913703C29757
:1042E000909337038093360368EC70E080E090E0B1
:1042F0000E94F3308091360390913703845F9140A0
:1043000024F4D0933703C093360380E195E069E548
:1043100071E00E94933580E195E06AE041E00E94FF
:10432000722F609136037091370380E195E04AE087
:1043300050E00E94803587E00E942D32892B09F0E1
:1043400090CF80E195E060E041E00E94722F80E133
:1043500095E060E071E00E94933580E195E060E0D7
:1043600041E00E94722F64E670E080E090E00E94DD
:10437000F33081E0809347056091360370913703F5
:1043800082E090E048C480E195E060E041E00E9476
:10439000722F80E195E063E971E00E94933511236B
:1043A00009F4BDC080E195E00E94A12F80E195E075
:1043B00060E040E00E94722F80E195E063E971E0E7
:1043C0000E94933580E195E060E041E00E94722F09
:1043D00080E195E06EE971E00E94933580E195E01F
:1043E00066E041E00E94722F6091290570912A05D4
:1043F00080E195E04AE050E00E94803566E970E097
:1044000080E090E00E94F330C9E0D0E086E00E94B6
:104410002D32892B79F58091290590912A050196F5
:1044200090932A058093290568EC70E080E090E085
:104430000E94F3308091290590912A050A9724F073
:10444000D0932A05C093290580E195E069E571E0E4
:104450000E94933580E195E066E041E00E94722F72
:104460006091290570912A0580E195E04AE050E0CD
:104470000E94803588E00E942D32892B79F5809149
:10448000290590912A05019790932A058093290583
:1044900068EC70E080E090E00E94F33080912905A4
:1044A00090912A0597FF04C010922A0510922905C1
:1044B00080E195E069E571E00E94933580E195E047
:1044C00066E041E00E94722F6091290570912A05F3
:1044D00080E195E04AE050E00E94803587E00E944C
:1044E0002D32892B09F092CF80E195E060E041E028
:1044F0000E94722F80E195E060E071E00E949335A8
:1045000080E195E060E041E00E94722F64E670E097
:1045100080E090E00E94F33081E080934705609155
:10452000290570912A0586E090E075C380E195E049
:1045300060E041E00E94722F80E195E064EA71E062
:104540000E949335112309F47BC080E195E00E941D
:10455000A12F80E195E060E040E00E94722F80E1B1
:1045600095E064EA71E00E94933580E195E060E0B7
:1045700041E00E94722F80913203909133030D9796
:1045800029F480E195E06CEA71E004C080E195E0F7
:104590006AEB71E00E94933566E970E080E090E09C
:1045A0000E94F33009E010E0CDE0D0E086E00E9408
:1045B0002D32892B81F480E195E060E041E00E949A
:1045C000722F80E195E06AEB71E00E9493351093C1
:1045D00033030093320388E00E942D32892B81F44B
:1045E00080E195E060E041E00E94722F80E195E07B
:1045F0006CEA71E00E949335D0933303C093320389
:1046000087E00E942D32892B89F680E195E060E0F9
:1046100041E00E94722F80E195E060E071E00E942D
:10462000933580E195E060E041E00E94722F64E6FE
:1046300070E080E090E00E94F33081E080934705D5
:1046400060913203709133038AE090E00E947A1EF9
:104650008DE060E00E94B33189E060E00E94B331F8
:104660008091320361E00E94B331D7C280E195E0CE
:1046700060E041E00E94722F80E195E068EC71E01B
:104680000E949335112309F479C080E195E00E94DE
:10469000A12F80E195E060E040E00E94722F80E170
:1046A00095E068EC71E00E94933580E195E060E070
:1046B00041E00E94722F80912B0590912C05892B4F
:1046C00029F480E195E063ED71E004C080E195E0BC
:1046D0006EED71E00E94933566E970E080E090E055
:1046E0000E94F330C1E0D0E088E00E942D32892B97
:1046F00081F480E195E060E041E00E94722F80E16A
:1047000095E063ED71E00E94933510922C051092B4
:104710002B0586E00E942D32892B81F480E195E003
:1047200060E041E00E94722F80E195E06EED71E063
:104730000E949335D0932C05C0932B0587E00E94EF
:104740002D32892B89F680E195E060E041E00E94FE
:10475000722F80E195E060E071E00E94933580E186
:1047600095E060E041E00E94722F64E670E080E036
:1047700090E00E94F33081E08093470560912B0523
:1047800070912C058CE090E046C280E195E060E0FD
:1047900041E00E94722F80E195E069EE71E00E9495
:1047A0009335112309F479C080E195E00E94A12F8F
:1047B00080E195E060E040E00E94722F80E195E0AA
:1047C00069EE71E00E94933580E195E060E041E0A0
:1047D0000E94722F80913C0390913D03892B29F414
:1047E00080E195E061EF71E004C080E195E06FEF5A
:1047F00071E00E94933566E970E080E090E00E94ED
:10480000F330C1E0D0E088E00E942D32892B81F4A2
:1048100080E195E060E041E00E94722F80E195E048
:1048200061EF71E00E94933510923D0310923C03BA
:1048300086E00E942D32892B81F480E195E060E0D2
:1048400041E00E94722F80E195E06FEF71E00E94DD
:104850009335D0933D03C0933C0387E00E942D32F3
:10486000892B89F680E195E060E041E00E94722F9B
:1048700080E195E060E071E00E94933580E195E091
:1048800060E041E00E94722F64E670E080E090E01A
:104890000E94F33081E08093470560913C03709162
:1048A0003D038EE090E0B7C180E195E060E041E03B
:1048B0000E94722F80E195E06DE072E00E949335D6
:1048C000112309F4BDC080E195E00E94A12F80E191
:1048D00095E060E040E00E94722F80E195E06DE09D
:1048E00072E00E94933580E195E060E041E00E9433
:1048F000722F80E195E06CE172E00E94933580E1D7
:1049000095E068E041E00E94722F60913E03709153
:104910003F0380E195E04AE050E00E94803566E97F
:1049200070E080E090E00E94F33086E00E942D323B
:10493000892B89F580913E0390913F0301969093D6
:104940003F0380933E0368EC70E080E090E00E94BB
:10495000F33080913E0390913F030B9734F08AE04F
:1049600090E090933F0380933E0380E195E069E5FA
:1049700071E00E94933580E195E068E041E00E949B
:10498000722F60913E0370913F0380E195E04AE011
:1049900050E00E94803588E00E942D32892B79F505
:1049A00080913E0390913F03019790933F03809342
:1049B0003E0368EC70E080E090E00E94F33080916C
:1049C0003E0390913F0397FF04C010923F03109263
:1049D0003E0380E195E069E571E00E94933580E156
:1049E00095E068E041E00E94722F60913E03709173
:1049F0003F0380E195E04AE050E00E94803587E087
:104A00000E942D32892B09F090CF80E195E060E083
:104A100041E00E94722F80E195E060E071E00E9429
:104A2000933580E195E060E041E00E94722F64E6FA
:104A300070E080E090E00E94F33081E080934705D1
:104A400060913E0370913F0382E190E0E4C080E119
:104A500095E060E041E00E94722F80E195E064E221
:104A600072E00E949335113009F0CBC080E195E0EF
:104A70000E94A12F80E195E060E040E00E94722F4B
:104A800080E195E064E272E00E94933580E195E078
:104A900060E041E00E94722F80E195E060E372E007
:104AA0000E94933580E195E06DE170E04AE050E0CE
:104AB0000E94803580E195E068E372E00E949335C2
:104AC00080E195E06DE041E00E94722F6091380531
:104AD0007091390580E195E04AE050E00E94803510
:104AE00066E970E080E090E00E94F330CDE1D0E034
:104AF00086E00E942D32892B79F5809138059091BE
:104B000039050196909339058093380568EC70E07B
:104B100080E090E00E94F330809138059091390553
:104B20004E9724F0D0933905C093380580E195E085
:104B300069E571E00E94933580E195E06DE041E028
:104B40000E94722F609138057091390580E195E0DF
:104B50004AE050E00E94803588E00E942D32892B87
:104B600079F5809138059091390501979093390531
:104B70008093380568EC70E080E090E00E94F330AC
:104B8000809138059091390597FF04C0109239053E
:104B90001092380580E195E069E571E00E94933557
:104BA00080E195E06DE041E00E94722F6091380550
:104BB0007091390580E195E04AE050E00E9480352F
:104BC00087E00E942D32892B09F092CF80E195E099
:104BD00060E041E00E94722F80E195E060E071E0CA
:104BE0000E94933580E195E060E041E00E94722FE1
:104BF00064E670E080E090E00E94F33081E0809312
:104C00004705109246051092450560913805709150
:104C1000390580E190E00E947A1EDF91CF911F91CB
:104C20000F910895EF92FF920F931F93CF93DF930D
:104C300080E195E00E94A12F80E195E060E040E0F6
:104C40000E94722F80E195E06BE372E00E94933541
:104C500086E00E942D32892B99F480914203909135
:104C60004303019690934303809342030C9744F0CF
:104C700081E090E090934303809342030E94B01838
:104C800088E00E942D32892B91F48091420390910B
:104C90004303019790934303809342031816190628
:104CA00034F08BE090E0909343038093420387E0DD
:104CB0000E942D32892B11F010E007C064E670E0ED
:104CC00080E090E00E94F33011E0809142039091E7
:104CD00043038630910509F421C487309105C4F45B
:104CE0008330910509F456C18430910544F4813034
:104CF000910539F1029711F00C94982EE9C0843097
:104D0000910509F433C2059711F00C94982E1AC33B
:104D10008930910509F4ABC68A3091054CF487308F
:104D2000910509F4E7C4089711F00C94982EBCC5BE
:104D30008A30910509F4EBC60B9711F00C94982E6C
:104D4000D0C780E195E060E041E00E94722F80E1F1
:104D500095E067E472E00E949335113009F0E8C7EE
:104D600080E195E00E94A12F80E195E060E040E0C5
:104D70000E94722F80E195E064E572E00E94933515
:104D80001092460510924505C1E0D0E098C080E140
:104D900095E06CE040E00E94722F80E195E0BE015A
:104DA0004AE050E00E94803580E195E061E040916A
:104DB00045050E94722F62E070E080E090E029E0FB
:104DC00030E040E050E00E9462386230710579F4D2
:104DD00060E070E080E090E027E430E040E050E008
:104DE0000E946238DC01CB010E94741D35C0633023
:104DF000710579F460E070E080E090E02FE630E04B
:104E000040E050E00E946238DC01CB010E944E1D60
:104E100023C06430710579F460E070E080E090E0D8
:104E20002FE630E040E050E00E946238DC01CB0128
:104E30000E94251D11C06530710574F060E070E0BE
:104E400080E090E027E831E040E050E00E946238E6
:104E5000DC01CB010E94FC1C809145059091460528
:104E60000197909346058093450580912B0590917D
:104E70002C05019719F587E00E942D32892BD9F76F
:104E80000E94B01868EE73E080E090E00E94F3307A
:104E900080E195E060E041E00E94722F80E195E0C2
:104EA00060E071E00E94933580E195E060E041E0D0
:104EB0000E94722F1092460510924505219680910E
:104EC0003A0390913B038C179D070CF060CF30C7DD
:104ED00080E195E060E041E00E94722F80E195E082
:104EE0006CE572E00E949335113009F021C780E132
:104EF00095E00E94A12F80E195E060E040E00E94F3
:104F0000722F80E195E069E672E00E94933510927D
:104F100046051092450580E195E06CE040E00E9476
:104F2000722F809138059091390597FF04C0109237
:104F3000390510923805609138057091390580E186
:104F400095E04AE050E00E94803580E195E061E024
:104F5000409145050E94722F809138059091390546
:104F60000E94D11C8091380590913905019690934B
:104F70003905809338054E9724F010923905109228
:104F80003805609138057091390580E190E00E9404
:104F90007A1ECEC680E195E060E041E00E94722F6B
:104FA00080E195E062E772E00E949335113009F0EC
:104FB000BFC680E195E00E94A12F80E195E060E00E
:104FC00040E00E94722F80E195E062E872E00E946A
:104FD0009335109246051092450501E010E0BDC0E2
:104FE00080E195E06CE040E00E94722F80E195E066
:104FF000B8014AE050E00E94803580E195E0609180
:10500000450541E00E94722F60E070E080E090E092
:1050100026E430E040E050E00E946238DC01CB0141
:105020007C010E94741D8091450590914605019771
:10503000909346058093450580912B0590912C0512
:10504000019709F088C0C0913803D09139032497A3
:1050500041C086E00E942D32892B59F40E94B0187D
:1050600068EE73E080E090E00E94F330C7010E9498
:10507000741D88E00E942D32892B31F50E94B018F2
:1050800068EE73E080E090E00E94F33080EB94E003
:10509000BE010E94A7386093340370933503609378
:1050A0002505709326052091340330913503C901FD
:1050B000880F991F820F931F9093280580932705CF
:1050C000C7010E94741D249768EC70E080E090E0B6
:1050D0000E94F33087E00E942D32892B09F0B9CF6E
:1050E0000E94B01868EE73E080E090E00E94F33018
:1050F000609138037091390380EB94E00E94A738E7
:1051000060933403709335036093250570932605EF
:105110002091340330913503C901880F991F820F04
:10512000931F909328058093270580E195E060E028
:1051300041E00E94722F80E195E060E071E00E9402
:10514000933580E195E060E041E00E94722F10927B
:105150004605109245050F5F1F4F80913A039091CD
:105160003B03801791070CF03BCFE2C580E195E04F
:1051700060E041E00E94722F80E195E06EE872E00D
:105180000E949335113009F0D3C580E195E00E946B
:10519000A12F80E195E060E040E00E94722F80E165
:1051A00095E06EE972E00E949335109246051092E8
:1051B000450501E010E0BDC080E195E06CE040E015
:1051C0000E94722F80E195E0B8014AE050E00E9411
:1051D000803580E195E06091450541E00E94722FA5
:1051E00060E070E080E090E02EE630E040E050E0EB
:1051F0000E946238DC01CB017C010E944E1D80912F
:105200004505909146050197909346058093450585
:1052100080912B0590912C05019709F088C0C091D1
:105220003803D0913903249741C086E00E942D3283
:10523000892B59F40E94B01868EE73E080E090E08A
:105240000E94F330C7010E944E1D88E00E942D325B
:10525000892B31F50E94B01868EE73E080E090E091
:105260000E94F33080EB94E0BE010E94A738609367
:1052700034037093350360932505709326052091C0
:10528000340330913503C901880F991F820F931F92
:105290009093280580932705C7010E944E1D2497EF
:1052A00068EC70E080E090E00E94F33087E00E94BC
:1052B0002D32892B09F0B9CF0E94B01868EE73E047
:1052C00080E090E00E94F3306091380370913903E0
:1052D00080EB94E00E94A738609334037093350309
:1052E0006093250570932605209134033091350392
:1052F000C901880F991F820F931F909328058093EF
:10530000270580E195E060E041E00E94722F80E196
:1053100095E060E071E00E94933580E195E060E007
:1053200041E00E94722F10924605109245050F5FD2
:105330001F4F80913A0390913B03801791070CF027
:105340003BCFF6C480E195E060E041E00E94722F1F
:1053500080E195E06AEA72E00E949335113009F02D
:10536000E7C480E195E00E94A12F80E195E060E034
:1053700040E00E94722F80E195E06AEB72E00E94AB
:105380009335109246051092450501E010E0BDC02E
:1053900080E195E06CE040E00E94722F80E195E0B2
:1053A000B8014AE050E00E94803580E195E06091CC
:1053B000450541E00E94722F60E070E080E090E0DF
:1053C0002EE630E040E050E00E946238DC01CB0184
:1053D0007C010E94251D809145059091460501970D
:1053E000909346058093450580912B0590912C055F
:1053F000019709F088C0C0913803D09139032497F0
:1054000041C086E00E942D32892B59F40E94B018C9
:1054100068EE73E080E090E00E94F330C7010E94E4
:10542000251D88E00E942D32892B31F50E94B0188D
:1054300068EE73E080E090E00E94F33080EB94E04F
:10544000BE010E94A73860933403709335036093C4
:105450002505709326052091340330913503C90149
:10546000880F991F820F931F90932805809327051B
:10547000C7010E94251D249768EC70E080E090E051
:105480000E94F33087E00E942D32892B09F0B9CFBA
:105490000E94B01868EE73E080E090E00E94F33064
:1054A000609138037091390380EB94E00E94A73833
:1054B000609334037093350360932505709326053C
:1054C0002091340330913503C901880F991F820F51
:1054D000931F909328058093270580E195E060E075
:1054E00041E00E94722F80E195E060E071E00E944F
:1054F000933580E195E060E041E00E94722F1092C8
:105500004605109245050F5F1F4F80913A03909119
:105510003B03801791070CF03BCF0AC480E195E074
:1055200060E041E00E94722F80E195E066EC72E05D
:105530000E949335113009F0FBC380E195E00E9491
:10554000A12F80E195E060E040E00E94722F80E1B1
:1055500095E064E572E00E94933510924605109242
:10556000450501E010E0BDC080E195E06CE040E061
:105570000E94722F80E195E0B8014AE050E00E945D
:10558000803580E195E06091450541E00E94722FF1
:1055900060E070E080E090E026E831E040E050E03C
:1055A0000E946238DC01CB017C010E94FC1C8091CE
:1055B00045059091460501979093460580934505D2
:1055C00080912B0590912C05019709F088C0C0911E
:1055D0003803D0913903249741C086E00E942D32D0
:1055E000892B59F40E94B01868EE73E080E090E0D7
:1055F0000E94F330C7010E94FC1C88E00E942D32FB
:10560000892B31F50E94B01868EE73E080E090E0DD
:105610000E94F33080EB94E0BE010E94A7386093B3
:10562000340370933503609325057093260520910C
:10563000340330913503C901880F991F820F931FDE
:105640009093280580932705C7010E94FC1C24978E
:1056500068EC70E080E090E00E94F33087E00E9408
:105660002D32892B09F0B9CF0E94B01868EE73E093
:1056700080E090E00E94F33060913803709139032C
:1056800080EB94E00E94A738609334037093350355
:1056900060932505709326052091340330913503DE
:1056A000C901880F991F820F931F9093280580933B
:1056B000270580E195E060E041E00E94722F80E1E3
:1056C00095E060E071E00E94933580E195E060E054
:1056D00041E00E94722F10924605109245050F5F1F
:1056E0001F4F80913A0390913B03801791070CF074
:1056F0003BCF1EC380E195E060E041E00E94722F45
:1057000080E195E065ED72E00E949335113009F07B
:105710000FC380E195E00E94A12F80E195E060E059
:1057200040E00E94722F80E195E065ED72E00E94FA
:105730009335109246051092450501E010E0ABC08C
:1057400080E195E06CE040E00E94722F80E195E0FE
:10575000B8014AE050E00E94803580E195E0609118
:10576000450541E00E94722F8DE295E00E94AB1B3F
:1057700080912B0590912C05019709F08AC0C0916A
:105780003803D0913903249743C086E00E942D321C
:10579000892B61F40E94B01868EE73E080E090E01D
:1057A0000E94F3308DE295E00E946A1C88E00E941E
:1057B0002D32892B39F50E94B01868EE73E080E035
:1057C00090E00E94F33080EB94E0BE010E94A73885
:1057D0006093340370933503609325057093260519
:1057E0002091340330913503C901880F991F820F2E
:1057F000931F90932805809327058DE295E00E94E2
:105800006A1C249768EC70E080E090E00E94F3301E
:1058100087E00E942D32892B09F0B7CF0E94B01883
:1058200068EE73E080E090E00E94F330609138030E
:105830007091390380EB94E00E94A73860933403A1
:1058400070933503609325057093260520913403EA
:1058500030913503C901880F991F820F931F9093D0
:1058600028058093270580E195E060E041E00E94F3
:10587000722F80E195E060E071E00E94933580E155
:1058800095E060E041E00E94722F10924605109270
:1058900045050F5F1F4F80913A0390913B0380179E
:1058A00091070CF04DCF44C280E195E060E041E00B
:1058B0000E94722F80E195E069EE71E00E949335BD
:1058C000113009F035C280E195E00E94A12F80E1FE
:1058D00095E060E040E00E94722F80E195E060EE8C
:1058E00072E00E949335109246051092450501E042
:1058F00010E0B4C080E195E06CE040E00E94722FBF
:1059000080E195E0B8014AE050E00E94803580E1F6
:1059100095E06091450541E00E94722F81E090E0A2
:105920000E94531B809145059091460501979093E5
:1059300046058093450580912B0590912C05019794
:1059400009F08AC0C0913803D0913903249743C02D
:1059500086E00E942D32892B61F40E94B01868EE17
:1059600073E080E090E00E94F3308AE395E00E94CB
:105970006A1C88E00E942D32892B39F50E94B018EC
:1059800068EE73E080E090E00E94F33080EB94E0FA
:10599000BE010E94A738609334037093350360936F
:1059A0002505709326052091340330913503C901F4
:1059B000880F991F820F931F9093280580932705C6
:1059C0008AE395E00E946A1C249768EC70E080E00E
:1059D00090E00E94F33087E00E942D32892B09F07D
:1059E000B7CF0E94B01868EE73E080E090E00E94AC
:1059F000F330609138037091390380EB94E00E949A
:105A0000A738609334037093350360932505709332
:105A100026052091340330913503C901880F991F61
:105A2000820F931F909328058093270580E195E0CE
:105A300060E041E00E94722F80E195E060E071E05B
:105A40000E94933580E195E060E041E00E94722F72
:105A500010924605109245050F5F1F4F80913A0343
:105A600090913B03801791070CF044CF61C180E116
:105A700095E060E041E00E94722F80E195E069EEE0
:105A800072E00E949335113009F052C180E195E037
:105A90000E94A12F80E195E060E040E00E94722F1B
:105AA00080E195E060EF72E00E9493351092460528
:105AB00010924505C1E0D0E022C080E195E06CE0A5
:105AC00040E00E94722F80E195E0BE014AE050E084
:105AD0000E94803580E195E06091450541E00E949B
:105AE000722F81E090E00E940A1B80914505909101
:105AF0004605019790934605809345052196809130
:105B00003A0390913B038C179D07BCF611C180E1CD
:105B100095E060E041E00E94722F80E195E069EF3E
:105B200072E00E949335113009F002C180E195E0E6
:105B30000E94A12F80E195E060E040E00E94722F7A
:105B400080E195E069EF72E00E94933580E195E095
:105B500060E041E00E94722F80E195E066E073E032
:105B60000E94933580E195E06AE041E00E94722F47
:105B7000609140037091410380E195E04AE050E07C
:105B80000E94803566E970E080E090E00E94F3308A
:105B900017E2E12EF12CC1E0D0E086E00E942D3228
:105BA000892B79F580914003909141030196909360
:105BB00041038093400368EC70E080E090E00E9435
:105BC000F3308091400390914103889724F0F09244
:105BD0004103E092400380E195E06FE073E00E94B2
:105BE000933580E195E06AE041E00E94722F609178
:105BF00040037091410380E195E04AE050E00E944B
:105C0000803588E00E942D32892B81F580914003F8
:105C1000909141030197909341038093400368EC76
:105C200070E080E090E00E94F3308091400390911A
:105C300041031816190624F0D0934103C093400382
:105C400080E195E06FE073E00E94933580E195E09C
:105C50006AE041E00E94722F60914003709141031D
:105C600080E195E04AE050E00E94803587E00E94A4
:105C70002D32892B11F010E013C080E195E060E037
:105C800041E00E94722F80E195E063E173E00E94A1
:105C9000933580E195E060E041E00E94722F11E0D1
:105CA000609140037091410388E090E00E947A1E69
:105CB000112309F472CF1092460510924505809188
:105CC0003A0390913B03BC01660F771F660F771F65
:105CD000680F791F80914003909141030E948A1CB4
:105CE00027C080E195E060E041E00E94722F80E1F2
:105CF00095E068E273E00E949335113089F468EC16
:105D000070E080E090E006C00E94971E64E670E0BC
:105D100080E090E00E94F330809147058823A1F352
:105D20001092470564E670E080E090E00E94F33056
:105D3000DF91CF911F910F91FF90EF9008950E94F6
:105D4000122664EB70E080E090E00E94F33008954A
:105D50000F931F938C01FC01868160E00E94D93172
:105D600081E090E00E944C31F801868161E00E9460
:105D7000D93181E090E00E944C31F801868160E0E9
:105D80000E94D93184E690E00E944C311F910F911E
:105D90000895CF92DF92EF92FF920F931F93CF93CC
:105DA000DF93D82EC92E282F392FC9018C01C0E0CE
:105DB000D0E0E62EFF24F801878161E00E94B33134
:105DC000B7010C2E02C0759567950A94E2F76170D1
:105DD000F80187810E94D93121960F5F1F4FC8308B
:105DE000D10549F78D2D9C2D0E94A82EDF91CF91D2
:105DF0001F910F91FF90EF90DF90CF900895CF9279
:105E0000DF92EF92FF920F931F93CF93DF93D82EE1
:105E1000C92E282F392FC9018C01C0E0D0E0E62E11
:105E2000FF24F801878161E00E94B331B7010C2E95
:105E300002C0759567950A94E2F76170F801878151
:105E40000E94D93121960F5F1F4FC430D10549F709
:105E50008D2D9C2D0E94A82EDF91CF911F910F9127
:105E6000FF90EF90DF90CF9008951F93CF93DF9333
:105E7000EC01162F8C81642F0E94D9318D818F3FC8
:105E800019F060E00E94D9318F8584FF05C0CE01F2
:105E9000612F0E94C92E0EC0612F70E084E07595BD
:105EA00067958A95E1F7CE010E94FF2ECE01612F02
:105EB0000E94FF2EDF91CF911F91089541E00E9433
:105EC000352F81E090E0089540E00E94352F08953D
:105ED000FC016089862F8460808B6C60CF010E94FA
:105EE000642F0895DF93CF93CDB7DEB728970FB611
:105EF000F894DEBF0FBECDBF9C01FE013196A7EF27
:105F0000B4E088E00D9001928150E1F7F9018389B6
:105F1000481710F0482F4150E42FF0E0EE0FFF1F1C
:105F2000EC0FFD1F8181680F6068C9010E94642F1A
:105F300028960FB6F894DEBF0FBECDBFCF91DF918C
:105F4000089561E00E94642F80ED97E00E944C313B
:105F50000895CF93DF93EC01423018F08F8588606D
:105F60008F874B8B1C8A222329F0413019F48F85AF
:105F700084608F8780E593EC0E944C318C8160E0D7
:105F80000E94D9318E8160E00E94D9318D818F3F8E
:105F900019F060E00E94D9316F8564FD1DC0CE010B
:105FA00063E00E94FF2E84E991E10E944C31CE0112
:105FB00063E00E94FF2E84E991E10E944C31CE0102
:105FC00063E00E94FF2E86E990E00E944C31CE01F2
:105FD00062E00E94FF2E16C06062CE010E94642F14
:105FE00084E991E10E944C316F856062CE010E948C
:105FF000642F86E990E00E944C316F856062CE018B
:106000000E94642F6F856062CE010E94642F84E03D
:10601000888BCE010E94682FCE010E94A12F82E0C2
:10602000898BCE0166E00E94642FDF91CF910895A5
:106030006F927F928F92AF92CF92EF920F931F93B6
:10604000DF93CF93CDB7DEB73C01162F842FF3013A
:10605000448325830683E782C086A18682869D8548
:1060600093879E8594879F8595879889968761E019
:106070000E94B331F30185818F3F19F061E00E94E6
:10608000B331F301868161E00E94B331112319F02D
:10609000F301178603C080E1F3018787C30160E144
:1060A00041E020E00E94A92FCF91DF911F910F9135
:1060B000EF90CF90AF908F907F906F9008958F92D8
:1060C000AF92CF92EF920F931F93CF93DF93DC01A8
:1060D000362F542F722F102FAE2C8C2C13961C920F
:1060E0001E92129783EF94E011969C938E9300D0AA
:1060F00000D0EDB7FEB73196CDB7DEB71982118269
:1061000012821382CD0161E0432F2FEF052FE72E7E
:10611000C12E0E9418300F900F900F900F90DF91BA
:10612000CF911F910F91EF90CF90AF908F900895E6
:10613000F999FECF72BD61BDF89A80B50895F999BD
:10614000FECF1FBA72BD61BD40BD0FB6F894FA9A7A
:10615000F99A0FBE08951F920F920FB60F92112455
:106160002F933F938F939F93AF93BF9380914D0550
:1061700090914E05A0914F05B09150053091510579
:106180000196A11DB11D232F2D5F2D3720F02D5716
:106190000196A11DB11D2093510580934D0590934B
:1061A0004E05A0934F05B0935005809149059091FD
:1061B0004A05A0914B05B0914C050196A11DB11D5A
:1061C0008093490590934A05A0934B05B0934C05E5
:1061D000BF91AF919F918F913F912F910F900FBEE3
:1061E0000F901F9018959B01AC017FB7F894809198
:1061F000490590914A05A0914B05B0914C0566B5B3
:10620000A89B05C06F3F19F00196A11DB11D7FBF6E
:10621000BA2FA92F982F8827860F911DA11DB11D78
:1062200062E0880F991FAA1FBB1F6A95D1F7BC01B6
:106230002DC0FFB7F8948091490590914A05A0912F
:106240004B05B0914C05E6B5A89B05C0EF3F19F092
:106250000196A11DB11DFFBFBA2FA92F982F882726
:106260008E0F911DA11DB11DE2E0880F991FAA1F7D
:10627000BB1FEA95D1F7861B970B885E9340C8F247
:10628000215030404040504068517C4F211531052D
:106290004105510571F60895019739F0880F991F4E
:1062A000880F991F02970197F1F70895789484B5A4
:1062B000826084BD84B5816084BD85B5826085BD02
:1062C00085B5816085BDEEE6F0E0808181608083E8
:1062D000E1E8F0E0108280818260808380818160CB
:1062E0008083E0E8F0E0808181608083E1EBF0E092
:1062F000808184608083E0EBF0E080818160808336
:10630000EAE7F0E08081846080838081826080831E
:106310008081816080838081806880831092C10049
:106320000895982F8E3008F09E5097708091ED045C
:106330008295880F880F807C892B80937C008091C8
:106340007A00806480937A0080917A0086FDFCCF89
:106350002091780040917900942F80E030E0282B44
:10636000392BC9010895482F50E0CA018552914D3B
:10637000FC0124914953514DFA0184918823C1F0C5
:10638000E82FF0E0EE0FFF1FE755F14DA591B49116
:10639000662341F49FB7F8948C91209582238C93C7
:1063A0009FBF08959FB7F8948C91822B8C939FBFC9
:1063B0000895482F50E0CA018151914DFC0124916C
:1063C000CA018552914DFC0194914953514DFA01F6
:1063D0003491332309F440C0222351F1233071F06A
:1063E000243028F42130A1F0223011F514C02630D9
:1063F000B1F02730C1F02430D9F404C0809180007E
:106400008F7703C0809180008F7D8093800010C0C3
:1064100084B58F7702C084B58F7D84BD09C080911B
:10642000B0008F7703C08091B0008F7D8093B00063
:10643000E32FF0E0EE0FFF1FED54F14DA591B49165
:106440002FB7F894662321F48C919095892302C08C
:106450008C91892B8C932FBF0895682F70E0CB010E
:106460008151914DFC012491CB018552914DFC014C
:1064700044916953714DFB019491992319F420E0E3
:1064800030E03CC0222351F1233071F0243028F455
:106490002130A1F0223011F514C02630B1F02730A0
:1064A000C1F02430D9F404C0809180008F7703C0FC
:1064B000809180008F7D8093800010C084B58F779D
:1064C00002C084B58F7D84BD09C08091B0008F77F4
:1064D00003C08091B0008F7D8093B000892F90E041
:1064E000880F991F8354914DFC01A591B4918C9113
:1064F00020E030E0842311F021E030E0C90108956C
:1065000008951F920F920FB60F9211242F933F936D
:106510004F938F939F93EF93FF934091C6002091E9
:106520009205309193052F5F3F4F2F73307080910C
:106530009405909195052817390759F0E091920537
:10654000F0919305EE5AFA4F4083309393052093D0
:106550009205FF91EF919F918F914F913F912F91D4
:106560000F900FBE0F901F901895E091E605F091E7
:10657000E705E05CFF4F8191919120813181821B81
:10658000930B8F739070892B11F00E9480320895C5
:106590001F920F920FB60F9211242F933F934F9398
:1065A0005F936F937F938F939F93AF93BF93EF937B
:1065B000FF932091D6053091D7058091D805909111
:1065C000D9052817390731F48091C1008F7D809358
:1065D000C10016C0E091D805F091D905EA56FA4FEE
:1065E00040818091D8059091D905019660E470E0D2
:1065F0000E94A7389093D9058093D8054093C60090
:10660000FF91EF91BF91AF919F918F917F916F918A
:106610005F914F913F912F910F900FBE0F901F9060
:106620001895AF92BF92DF92EF92FF920F931F9354
:10663000CF93DF93EC017A018B01DD24403081EEB2
:10664000580780E0680780E0780711F0DD24D394D4
:1066500091E0A92EB12CEC89FD89DD2069F0C501FE
:106660000E8C02C0880F991F0A94E2F7808360E0C5
:1066700079E08DE390E005C0108260E874E88EE177
:1066800090E0A80197010E94BA3821503040404064
:106690005040569547953795279580E1203038072B
:1066A00020F0DD2011F0DD24D6CFE889F989308390
:1066B000EA89FB892083EE89FF89408121E030E06F
:1066C000C9010A8C02C0880F991F0A94E2F7482B6F
:1066D0004083EE89FF894081C9010B8C02C0880F7D
:1066E000991F0A94E2F7482B4083EE89FF89408185
:1066F000C9010C8C02C0880F991F0A94E2F7482B3D
:106700004083EE89FF8980810D8C02C0220F331FE8
:106710000A94E2F7209528232083DF91CF911F91DF
:106720000F91FF90EF90DF90BF90AF900895DC0144
:106730001C96ED91FC911D97E05CFF4F21913191EA
:1067400080819181281B390B2F733070C901089506
:10675000DC011C96ED91FC911D97E05CFF4F2081C0
:106760003181E054F040DF01AE5BBF4F8D919C91D1
:1067700011972817390719F42FEF3FEF07C08D91B4
:106780009C91E80FF91F8081282F30E0C9010895FE
:10679000DC011C96ED91FC911D97E05CFF4F208180
:1067A0003181E054F040DF01AE5BBF4F8D919C9191
:1067B00011972817390719F42FEF3FEF10C08D916B
:1067C0009C911197E80FF91F20818D919C91119751
:1067D00001968F73907011969C938E9330E0C9014F
:1067E0000895FC0186859785DC01A05CBF4FFC0104
:1067F000EE5BFF4F2D913C9111978081918128177D
:106800003907C1F70895CF93DF93EC01462FEE854A
:10681000FF85E05CFF4F80819181E054F04001965C
:1068200060E470E00E94A7389C01DF01AE5BBF4FBF
:106830008D919C91119728173907D1F3E05CFF4F98
:1068400080819181E054F040E80FF91F4083EE858C
:10685000FF85E05CFF4F31832083EE89FF89208133
:1068600081E090E00D8C02C0880F991F0A94E2F736
:10687000282B208381E090E0DF91CF910895109242
:10688000DD051092DC0588EE93E0A0E0B0E0809397
:10689000DE059093DF05A093E005B093E10583E06A
:1068A00095E09093DB058093DA0582E595E090937F
:1068B000E7058093E60586E995E09093E9058093E6
:1068C000E80585EC90E09093EB058093EA0584EC75
:1068D00090E09093ED058093EC0580EC90E0909330
:1068E000EF058093EE0581EC90E09093F1058093A5
:1068F000F00586EC90E09093F3058093F20584E038
:106900008093F40583E08093F50587E08093F60596
:1069100085E08093F70581E08093F8050895CF9393
:10692000DF930E9456310E940A1EC5EBD2E30E94FB
:106930009F2E2097E1F30E94B532F9CFCF92DF92DC
:10694000EF92FF920F931F93CF93DF937C016B0124
:106950008A01C0E0D0E00FC0D6016D916D01D70172
:10696000ED91FC910190F081E02DC7010995C80FD0
:10697000D91F015010400115110571F7CE01DF91AB
:10698000CF911F910F91FF90EF90DF90CF900895DE
:10699000CF93DF93DB010D900020E9F71197A61B41
:1069A000B70BEC01E881F9810280F381E02DAD01A4
:1069B0000995DF91CF9108954F925F927F928F92C8
:1069C0009F92AF92BF92CF92DF92EF92FF920F937E
:1069D0001F93DF93CF93CDB7DEB7A1970FB6F8948F
:1069E000DEBF0FBECDBF2C01742ECB01223008F4C8
:1069F0002AE019A231E2C32ED12CCC0EDD1E822E4C
:106A00009924AA24BB24672D752FA50194010E9407
:106A1000BA3879018A01C801B701A50194010E9421
:106A20008838472D461B0894C108D1084A3014F411
:106A3000405D01C0495CF6014083E114F1040105A9
:106A4000110521F07E2C5F2DC801DDCFC201B601FA
:106A50000E94C834A1960FB6F894DEBF0FBECDBF1A
:106A6000CF91DF911F910F91FF90EF90DF90CF902A
:106A7000BF90AF909F908F907F905F904F900895C0
:106A8000CF92DF92EF92FF920F931F93CF93DF93FA
:106A9000EC016A017B012115310541F4E881F9819E
:106AA0000190F081E02D642F09951FC02A30310537
:106AB000D1F477FF17C0E881F9810190F081E02DD2
:106AC0006DE209958C0144275527BA014C195D09DF
:106AD0006E097F09CE012AE00E94DC349801280F5C
:106AE000391F04C02AE00E94DC349C01C901DF91F7
:106AF000CF911F910F91FF90EF90DF90CF9008956D
:106B0000EF92FF920F931F937B019A010027F7FCEE
:106B10000095102FB801A7010E9440351F910F91D9
:106B2000FF90EF9008950E94C8340895813041F09D
:106B3000813018F08230D1F409C010926E000895AF
:106B400080916F008D7F80936F0008958091700019
:106B50008D7F8093700081E08093B0008091B100C0
:106B6000887F84608093B1001092B30008951F93D2
:106B7000182F8091EE04811711F09FEF06C0E3E01B
:106B8000FFE294918FEF8093EE04892F0E94963557
:106B9000812F60E00E94D9311F9108951F920F92BA
:106BA0000FB60F9211242F933F934F935F936F93E0
:106BB0007F938F939F93AF93BF93EF93FF938091B6
:106BC000070690910806A0910906B0910A06009761
:106BD000A105B10551F1E0910B06F0910C06808101
:106BE00090910D0689278083809107069091080671
:106BF000A0910906B0910A06181619061A061B0676
:106C0000C4F48091070690910806A0910906B091FE
:106C10000A060197A109B109809307069093080617
:106C2000A0930906B0930A0604C08091EE040E9466
:106C3000B735FF91EF91BF91AF919F918F917F9168
:106C40006F915F914F913F912F910F900FBE0F90D9
:106C50001F9018952F923F925F926F927F928F9222
:106C60009F92AF92BF92CF92DF92EF92FF920F93DB
:106C70001F93DF93CF9300D000D0CDB7DEB7A82FFE
:106C80001B0129833A834B835C838091EE048A172E
:106C900021F4E3E0FFE2549082C08F3F09F0DAC1B3
:106CA000A093EE04E3E0FFE254902FEF521609F4B4
:106CB000D1C181E0581639F192E0591609F449C062
:106CC000552009F06CC014BC15BC84B5826084BD2D
:106CD00085B5816085BD2A2F30E0F901E953F14D7A
:106CE000E491F0E0EE0FFF1FED54F14D859194918A
:106CF0009093FE058093FD052552314DF901849155
:106D00008093FF054EC01092800010928100809108
:106D100081008860809381008091810081608093F0
:106D200081002A2F30E0F901E953F14DE491F0E0C0
:106D3000EE0FFF1FED54F14D859194919093050650
:106D4000809304062552314DF90184918093060603
:106D500028C01092B0001092B1008091B000826003
:106D60008093B0008091B10081608093B1002A2FA0
:106D700030E0F901E953F14DE491F0E0EE0FFF1F2F
:106D8000ED54F14D8591949190930C0680930B06F0
:106D90002552314DF901849180930D0602C057FCB4
:106DA00059C18A2F61E00E94B331552021F0F2E0F1
:106DB0005F1609F0BEC031018824992460E072E1B9
:106DC0008AE790E0A40193010E94DC3859016A012E
:106DD000860175010894E108F108010911092FEFF6
:106DE000E216F1040105110509F008F499C060E408
:106DF00072E48FE090E0A40193010E94DC387901F5
:106E00008A010894E108F1080109110982E0581685
:106E1000C1F49FEFE916F1040105110509F008F42A
:106E200084C060E970ED83E090E0A40193010E94CA
:106E3000DC3879018A010894E108F1080109110997
:106E400083E0AFEFEA16F1040105110509F008F43B
:106E500068C068E478EE81E090E0A40193010E94AC
:106E6000DC3879018A010894E108F1080109110967
:106E7000552011F483E01DC0B2E05B1611F084E0F0
:106E800018C0EFEFEE16F1040105110509F008F442
:106E9000DFC064E274EF80E090E0A40193010E94FF
:106EA000DC3879018A010894E108F1080109110927
:106EB00085E0FFEFEF16F1040105110591F188F16E
:106EC00062E17AE780E090E0A40193010E94DC385F
:106ED00079018A010894E108F10801091109552096
:106EE00011F086E001C084E02FEFE216F104010505
:106EF0001105B9F0B0F0C601B50120E034E040E082
:106F000050E00E94DC3879018A010894E108F10818
:106F100001091109552011F087E008C085E003C080
:106F200081E0552019F485BD3AC082E08093B1001C
:106F300036C05101CC24DD2460E072E18AE790E0A4
:106F4000A60195010E94DC3879018A010894E108C4
:106F5000F1080109110980E0E81680E0F80681E0F7
:106F6000080780E0180710F491E010C068E478EE9C
:106F700081E090E0A60195010E94DC3879018A0148
:106F80000894E108F1080109110993E0A1E05A16FB
:106F900031F480918100887F982B909381008981C2
:106FA0009A81AB81BC810097A105B10529F48FEFCF
:106FB0009FEFAFEFBFEF13C0220C331CB10180E095
:106FC00090E029813A814B815C810E94883828EECB
:106FD00033E040E050E00E94BA38C901DA01E1E054
:106FE0005E16A1F0F2E05F1619F1552099F5E7BCA5
:106FF0008093F9059093FA05A093FB05B093FC05E7
:1070000080916E00826080936E0024C0F0928900AF
:10701000E09288008093000690930106A0930206F8
:10702000B093030680916F00826080936F0012C05E
:10703000E092B3008093070690930806A093090698
:10704000B0930A068091700082608093700002C045
:1070500084E06CCF0F900F900F900F90CF91DF9145
:107060001F910F91FF90EF90DF90CF90BF90AF9066
:107070009F908F907F906F905F903F902F9008959A
:10708000EF92FF920F931F937B018C0161157105A5
:107090008105910529F420E030E040E050E00BC08C
:1070A0000E940118A80197010E94DC38AC01CB01B5
:1070B000DA019C01AD01B901CA011F910F91FF9046
:1070C000EF900895EF92FF920F931F937B018C0135
:1070D000621773078407950764F4261B370B480B68
:1070E000590BCA01B9010E944038E60EF71E081F6D
:1070F000191FB701C8011F910F91FF90EF900895DC
:10710000009729F0BC0180E090E00E9406180895E5
:10711000629FD001739FF001829FE00DF11D649F7B
:10712000E00DF11D929FF00D839FF00D749FF00D07
:10713000659FF00D9927729FB00DE11DF91F639FA8
:10714000B00DE11DF91FBD01CF011124089597FB7A
:10715000092E07260AD077FD04D049D006D000209A
:107160001AF4709561957F4F0895F6F79095819583
:107170009F4F0895A1E21A2EAA1BBB1BFD010DC053
:10718000AA1FBB1FEE1FFF1FA217B307E407F507D7
:1071900020F0A21BB30BE40BF50B661F771F881FB3
:1071A000991F1A9469F760957095809590959B0149
:1071B000AC01BD01CF01089597FB092E05260ED025
:1071C00057FD04D0D7DF0AD0001C38F45095409505
:1071D000309521953F4F4F4F5F4F0895F6F79095AB
:1071E0008095709561957F4F8F4F9F4F0895AA1B93
:1071F000BB1B51E107C0AA1FBB1FA617B70710F0A2
:10720000A61BB70B881F991F5A95A9F780959095D3
:10721000BC01CD010895EE0FFF1F0590F491E02D04
:1072200009942F923F924F925F926F927F928F922A
:107230009F92AF92BF92CF92DF92EF92FF920F9305
:107240001F93CF93DF93CDB7DEB7CA1BDB0B0FB60F
:10725000F894DEBF0FBECDBF09942A8839884888CC
:107260005F846E847D848C849B84AA84B984C88462
:10727000DF80EE80FD800C811B81AA81B981CE0F59
:10728000D11D0FB6F894DEBF0FBECDBFED0108953E
:10729000F894FFCF20202020202020202020202014
:1072A000202020200043572D506172746E6572209B
:1072B0000056312E3330005665722E203332382C72
:1072C00020444C384B464F3B0053657475703A0070
:1072D000476573636877696E6469676B6569740095
:1072E00057504D202831302D3630293A00202000CB
:1072F00044757263686761656E6765002832352D75
:10730000353030293A00546F6E686F6568650054F7
:107310006F6E686F6568652028487A2900353030BF
:107320002D313230303A004661726E73776F72746D
:107330006800446F74733A0041757367616E67004B
:107340002020202020202065787465726E00202087
:107350002020202020696E7465726E00496E74656D
:1073600072616B74697600202020202020206175D6
:1073700073002020202020202065696E0047727550
:107380007070656E002020202020202020202041C9
:107390002D5A002020202020412D5A2C20302D391C
:1073A00000416E7A61686C205A65696368656E0099
:1073B000416E7A61686C3A0051534F2D4175737775
:1073C00061686C0051534F2028302D00293A004845
:1073D000617570746D656E75653A00576F7274747F
:1073E0007261696E696E6700576F727465203A004A
:1073F00051534F2D547261696E696E670051534F3E
:10740000204E722E3A00576F7274652032205A65F2
:10741000696368656E00576F72746520322042534D
:107420003A00576F7274652033205A656963686546
:107430006E00576F72746520332042533A00576FC5
:107440007274652034205A65696368656E00576FF1
:1074500072746520342042533A004C61656E676552
:10746000726520576F727465005275667A6569633C
:1074700068656E004772757070656E3A0052656996
:1074800068656E0052656968656E203A004B6F63EF
:10749000682D4D6574686F64650028312D33392976
:1074A0003A20002020200020202020202020202002
:1074B00020202020202020202020200053657475CB
:1074C0007000010000000D003C008A021400320030
:1074D0000100050001000100010033683B00006469
:1074E0006B3B0000646C3B0000346F3B0000356177
:1074F0003B000036643B000039683B0000613B0004
:10750000000063623B0000636B3B0000636E3B0066
:107510000063743B000064363B0000646A3B00007B
:1075200065613B000065613B000065693B000065EB
:10753000733B0000663B00000066793B0000673B40
:10754000000000676E3B000068323B000068613B52
:10755000000068623B000068763B0000693B000069
:10756000006A343B00006B3B0000006D3B000000F4
:107570006E3B0000006F6B3B00006F6E3B00006FC6
:107580007A3B000070613B000070643B0000733583
:107590003B000073763B000074393B000074613B94
:1075A000000075613B0000756E3B000075723B008A
:1075B0000076723B0000773B00000078613B0000E2
:1075C00078763B0000796F3B00007A333B00007A0D
:1075D0006C3B00007A703B00007A723B00007A76C8
:1075E0003B000074663B000076753B000076733606
:1075F0003B006A613B000078653B00007A733B000A
:10760000006C613B00006B3B006D3B00753B007202
:107610003B00653B00733B006E3B00613B00703BF1
:1076200000743B006C3B00773B00693B002E3B0045
:107630006A3B007A3B00663B006F3B00793B002CC5
:107640003B00763B00673B00353B002F3B00713B26
:1076500000393B00323B00683B00333B00383B00C5
:10766000623B003F3B00343B00373B00633B003153
:107670003B00643B00363B00303B00783B003D3B29
:107680000001FF000000005E2F9E34000040001447
:107690000054000000000003349E349733C833A820
:1076A00033F13300FFFFFFFFFFFFFFFFFFFFFFFF8F
:1076B000FFFFFFFFFFFFFFFFFFFFFFFFFFFFFFFFDA
:1076C000FFFFFFFFFFFFFFFFFFFFFFFFFFFFFFFFCA
:1076D000FFFFFFFFFFFFFFFFFFFFFFFFFFFFFFFFBA
:1076E000FFFFFFFFFFFFFFFFFFFFFFFFFFFFFFFFAA
:1076F000FFFFFFFFFFFFFFFFFFFFFFFFFFFFFFFF9A
:10770000FFFFFFFFFFFFFFFFFFFFFFFFFFFFFFFF89
:10771000FFFFFFFFFFFFFFFFFFFFFFFFFFFFFFFF79
:10772000FFFFFFFFFFFFFFFFFFFFFFFFFFFFFFFF69
:10773000FFFFFFFFFFFFFFFFFFFFFFFFFFFFFFFF59
:10774000FFFFFFFFFFFFFFFFFFFFFFFFFFFFFFFF49
:10775000FFFFFFFFFFFFFFFFFFFFFFFFFFFFFFFF39
:10776000FFFFFFFFFFFFFFFFFFFFFFFFFFFFFFFF29
:10777000FFFFFFFFFFFFFFFFFFFFFFFFFFFFFFFF19
:10778000FFFFFFFFFFFFFFFFFFFFFFFFFFFFFFFF09
:10779000FFFFFFFFFFFFFFFFFFFFFFFFFFFFFFFFF9
:1077A000FFFFFFFFFFFFFFFFFFFFFFFFFFFFFFFFE9
:1077B000FFFFFFFFFFFFFFFFFFFFFFFFFFFFFFFFD9
:1077C000FFFFFFFFFFFFFFFFFFFFFFFFFFFFFFFFC9
:1077D000FFFFFFFFFFFFFFFFFFFFFFFFFFFFFFFFB9
:1077E000FFFFFFFFFFFFFFFFFFFFFFFFFFFFFFFFA9
:1077F000FFFFFFFFFFFFFFFFFFFFFFFFFFFFFFFF99
:107800000C94343C0C94513C0C94513C0C94513CE1
:107810000C94513C0C94513C0C94513C0C94513CB4
:107820000C94513C0C94513C0C94513C0C94513CA4
:107830000C94513C0C94513C0C94513C0C94513C94
:107840000C94513C0C94513C0C94513C0C94513C84
:107850000C94513C0C94513C0C94513C0C94513C74
:107860000C94513C0C94513C11241FBECFEFD8E036
:10787000DEBFCDBF11E0A0E0B1E0ECE9FFE702C060
:1078800005900D92A230B107D9F712E0A2E0B1E065
:1078900001C01D92AD30B107E1F70E942D3D0C945F
:1078A000CC3F0C94003C982F959595959595959582
:1078B000905D8F708A307CF0282F295A8091C0000B
:1078C00085FFFCCF9093C6008091C00085FFFCCF60
:1078D0002093C6000895282F205DF0CF982F809127
:1078E000C00085FFFCCF9093C6000895EF92FF92F1
:1078F0000F931F93EE24FF2487018091C00087FD22
:1079000017C00894E11CF11C011D111D81E4E8164B
:1079100082E4F8068FE0080780E0180770F3E09132
:107920000401F091050109958091C00087FFE9CF1E
:107930008091C6001F910F91FF90EF9008950E94D3
:10794000763C982F8091C00085FFFCCF9093C600B5
:1079500091362CF490330CF09053892F089597555D
:10796000892F08951F930E949F3C182F0E949F3CCF
:107970001295107F810F1F9108951F93182F882350
:1079800021F00E94763C1150E1F71F9108951F935A
:10799000182F0E94763C803249F0809103018F5F5E
:1079A000809303018530C1F01F9108958091C0003C
:1079B00085FFFCCF84E18093C6008091C00085FFE5
:1079C000FCCF1093C6008091C00085FFFCCF80E102
:1079D0008093C6001F910895E0910401F091050184
:1079E00009951F9108950E94763C803241F0809164
:1079F00003018F5F80930301853081F008958091AA
:107A0000C00085FFFCCF84E18093C6008091C00058
:107A100085FFFCCF80E18093C6000895E0910401CA
:107A2000F09105010995089540E951E08823A1F0FE
:107A30002D9A28EE33E0FA013197F1F721503040CA
:107A4000D1F72D9828EE33E0FA013197F1F7215064
:107A50003040D1F7815061F708953F924F925F9285
:107A60006F927F928F929F92AF92BF92CF92DF924E
:107A7000EF92FF920F931F93CF93DF93000080E16B
:107A80008093C4001092C50088E18093C10086E015
:107A90008093C2005098589A259A81E00E94143D24
:107AA00024E1F22E9EE1E92E85E9D82E0FE0C02ECA
:107AB00010E1B12EAA24A394B1E49B2EA6E58A2E50
:107AC000F2E57F2EE0E26E2E79E4572E63E5462E36
:107AD00050E5352E0E94763C8033B1F18133B9F107
:107AE000803409F46FC0813409F476C0823409F41B
:107AF00085C0853409F488C0803531F1823521F1A3
:107B0000813511F1853509F485C0863509F48DC0BC
:107B1000843609F496C0843709F403C1853709F423
:107B200072C1863709F466C0809103018F5F80932C
:107B30000301853079F6E0910401F0910501099582
:107B40000E94763C803351F60E94F33CC3CF0E94E2
:107B5000763C803249F78091C00085FFFCCFF092DF
:107B6000C6008091C00085FFFCCF9092C600809136
:107B7000C00085FFFCCF8092C6008091C00085FFC9
:107B8000FCCF7092C6008091C00085FFFCCF609250
:107B9000C6008091C00085FFFCCF5092C600809146
:107BA000C00085FFFCCF4092C6008091C00085FFD9
:107BB000FCCF3092C6008091C00085FFFCCFB09210
:107BC000C60088CF0E94763C863808F4BDCF0E945C
:107BD000763C0E94F33C7ECF0E94763C803809F4CC
:107BE0009CC0813809F40BC1823809F43CC1883942
:107BF00009F48FC080E00E94C73C6CCF84E10E94F2
:107C0000BD3C0E94F33C66CF85E00E94BD3C0E94D3
:107C1000F33C60CF0E94763C809306010E94763C44
:107C2000809307010E94F33C55CF0E94763C80333D
:107C300009F41DC183E00E94BD3C80E00E94C73C66
:107C400049CF0E94763C809309020E94763C809343
:107C5000080280910C028E7F80930C020E94763C79
:107C6000853409F415C18091080290910902892B8D
:107C700089F000E010E00E94763CF801E85FFE4FDA
:107C800080830F5F1F4F80910802909109020817AF
:107C9000190788F30E94763C803209F045CF809125
:107CA0000C0280FF01C16091060170910701660F0F
:107CB000771F7093070160930601A0910802B091AD
:107CC00009021097C9F0E8E0F1E09B01AD014E0F09
:107CD0005F1FF999FECF32BD21BD819180BDFA9A17
:107CE000F99A2F5F3F4FE417F50799F76A0F7B1F4B
:107CF00070930701609306018091C00085FFFCCF5F
:107D0000F092C6008091C00085FFFCCFB092C60003
:107D1000E1CE83E00E94C73CDDCE82E00E94C73CFA
:107D2000D9CE0E94763C809309020E94763C8093D3
:107D300008028091060190910701880F991F909386
:107D40000701809306010E94763C853409F4A6C0A1
:107D500080910C028E7F80930C020E94763C8032D0
:107D600009F0B8CE8091C00085FFFCCFF092C6002C
:107D7000609108027091090261157105B9F140E046
:107D800050E080910C02A82FA170B82FB27011C0E2
:107D9000BB2309F45CC0E0910601F0910701319624
:107DA000F0930701E09306014F5F5F4F46175707B7
:107DB000E8F4AA2369F3F999FECF209106013091E6
:107DC000070132BD21BDF89A90B58091C00085FFB2
:107DD000FCCF9093C6002F5F3F4F30930701209355
:107DE00006014F5F5F4F4617570718F38091C00099
:107DF00085FDE5CE8091C00085FFF8CFE0CE81E023
:107E00000E94C73C67CE0E94763C803209F08CCE3F
:107E10008091C00085FFFCCFF092C6008091C00029
:107E200085FFFCCFE092C6008091C00085FFFCCFAB
:107E3000D092C6008091C00085FFFCCFC092C600E2
:107E40008091C00085FFFCCFB092C60043CEE09188
:107E50000601F091070194918091C00085FFFCCF4D
:107E60009093C6009CCF80E10E94C73C33CE0E9415
:107E7000763C0E94763C182F0E94763C112309F430
:107E800083C0113009F484C08FE00E94C73C22CE29
:107E900080910C02816080930C02E5CE80910C02EF
:107EA000816080930C0259CF809107018823880F4D
:107EB000880B8A2180930B02809106019091070123
:107EC000880F991F90930701809306018091080203
:107ED00080FF09C080910802909109020196909359
:107EE000090280930802F894F999FECF1127E091D6
:107EF0000601F0910701C8E0D1E08091080290915D
:107F00000902103091F40091570001700130D9F34B
:107F100003E000935700E89500915700017001308D
:107F2000D9F301E100935700E89509901990009169
:107F3000570001700130D9F301E000935700E89534
:107F40001395103498F011270091570001700130FB
:107F5000D9F305E000935700E895009157000170B0
:107F60000130D9F301E100935700E895329602976A
:107F700009F0C7CF103011F00296E5CF112480919F
:107F8000C00085FFB9CEBCCE8EE10E94C73CA2CD19
:0E7F900085E90E94C73C9ECDF894FFCF80008B
:00000001FF
